 esai_wm8580

 Timestamp is 4fb05c77 (Mon May 14 13:14:31 2012)

 Preferred load address is 10000000

 Start         Length     Name                   Class
 0001:00000000 000031eaH .rdata                  CODE
 0001:000031ec 00000028H .rdata$debug            CODE
 0001:00003214 00012680H .text                   CODE
 0001:00015894 0000003cH .xdata                  CODE
 0001:000158d0 00000064H .idata$2                CODE
 0001:00015934 00000014H .idata$3                CODE
 0001:00015948 0000010cH .idata$4                CODE
 0001:00015a54 00000188H .idata$6                CODE
 0001:00015be0 0000009bH .edata                  CODE
 0002:00000000 0000010cH .idata$5                DATA
 0002:00000110 0000054cH .data                   DATA
 0002:0000065c 00000020H .bss                    DATA
 0003:00000000 00000b60H .pdata                  DATA

  Address         Publics by Value              Rva+Base       Lib:Object

 0000:00000000       ___safe_se_handler_count   00000000     <absolute>
 0000:00000000       ___safe_se_handler_table   00000000     <absolute>
 0001:00000020       ??_C@_1FE@GFEFLFNN@?$AAC?$AAr?$AAe?$AAa?$AAt?$AAe?$AA?5?$AAC?$AAS?$AAP?$AAI?$AA?5?$AAf?$AAi?$AAl?$AAe?$AA?5?$AAh?$AAa?$AAn?$AAd?$AAl?$AAe?$AA?5?$AAf?$AAa?$AAi?$AAl?$AAe?$AAd?$AA?5?$AAe@ 10001020     wm8580.obj
 0001:00000074       ??_C@_1M@BALJCCCP@?$AAS?$AAP?$AAI?$AA1?$AA?3?$AA?$AA@ 10001074     wm8580.obj
 0001:00000080       ??_C@_1DC@CIKBPPAF@?$AAR?$AAe?$AAa?$AAd?$AA?5?$AAW?$AAM?$AA8?$AA5?$AA8?$AA0?$AA?5?$AAR?$AAE?$AAG?$AA?5?$AAF?$AAa?$AAi?$AAl?$AAe?$AAd?$AA?$AN?$AA?6?$AA?$AA@ 10001080     wm8580.obj
 0001:000000b4       ??_C@_1DA@FKDIIMJ@?$AAW?$AAr?$AAi?$AAt?$AAe?$AA?5?$AAW?$AAM?$AA8?$AA5?$AA8?$AA0?$AA?5?$AAR?$AAE?$AAG?$AA?5?$AAF?$AAa?$AAi?$AAl?$AAe?$AAd?$AA?$AA@ 100010b4     wm8580.obj
 0001:000000e8       ??_C@_1EE@JPIDNDCG@?$AA?$CF?$AAs?$AA?3?$AA?5?$AAS?$AAe?$AAt?$AA?5?$AAI?$AA2?$AAC?$AA?5?$AAm?$AAa?$AAs?$AAt?$AAe?$AAr?$AA?5?$AAm?$AAo?$AAd?$AAe?$AA?5?$AAf?$AAa?$AAi?$AAl?$AAe?$AAd?$AA?$CB?$AA?$AN@ 100010e8     ak5702.obj
 0001:0000012c       ??_C@_1DM@DLGOCCCK@?$AA?$CF?$AAs?$AA?3?$AA?5?$AAO?$AAp?$AAe?$AAn?$AA?5?$AAI?$AA2?$AAC?$AA?5?$AAh?$AAa?$AAn?$AAd?$AAl?$AAe?$AA?5?$AAf?$AAa?$AAi?$AAl?$AAe?$AAd?$AA?$CB?$AA?$AN?$AA?6?$AA?$AA@ 1000112c     ak5702.obj
 0001:00000168       ??_C@_1CC@PFAOBHLH@?$AAC?$AAA?$AAK?$AA5?$AA7?$AA0?$AA2?$AA?3?$AA?3?$AAC?$AAA?$AAK?$AA5?$AA7?$AA0?$AA2?$AA?$AA@ 10001168     ak5702.obj
 0001:0000018c       ??_C@_1CI@OHCJFJPM@?$AAE?$AAR?$AAR?$AAO?$AAR?$AA?3?$AA?5?$AA?$CF?$AAs?$AA?5?$AAl?$AAi?$AAn?$AAe?$AA?5?$AA?$CF?$AAd?$AA?3?$AA?5?$AA?$AA@ 1000118c     ak5702.obj
 0001:000001b8       ??_C@_1JE@KNGJCFGP@?$AAC?$AA?3?$AA?2?$AAW?$AAI?$AAN?$AAC?$AAE?$AAR?$AAO?$AAO?$AAT?$AAS?$AA?2?$AAT?$AAo?$AAp?$AAa?$AAz?$AA?2?$AAW?$AAI?$AAN?$AAC?$AAE?$AA6?$AA0?$AA0?$AA?2?$AAP?$AAL?$AAA@ 100011b8     ak5702.obj
 0001:0000024c       ??_C@_1M@LCEEOPDH@?$AAI?$AA2?$AAC?$AA1?$AA?3?$AA?$AA@ 1000124c     ak5702.obj
 0001:00000258       ??_C@_1HE@MIOBJJKD@?$AA?$CF?$AAs?$AA?3?$AA?5?$AAR?$AAe?$AAa?$AAd?$AA?5?$AAA?$AAK?$AA5?$AA7?$AA0?$AA2?$AA?5?$AAr?$AAe?$AAg?$AAi?$AAs?$AAt?$AAe?$AAr?$AA?5?$AA0?$AAx?$AA?$CF?$AAx?$AA?5?$AAf?$AAa@ 10001258     ak5702.obj
 0001:000002cc       ??_C@_1CM@PJAEHAOL@?$AAC?$AAA?$AAK?$AA5?$AA7?$AA0?$AA2?$AA?3?$AA?3?$AAR?$AAe?$AAa?$AAd?$AAR?$AAe?$AAg?$AAi?$AAs?$AAt?$AAe?$AAr?$AA?$AA@ 100012cc     ak5702.obj
 0001:000002f8       ??_C@_1GO@EIPNEGLA@?$AA?$CF?$AAs?$AA?3?$AA?5?$AAW?$AAr?$AAi?$AAt?$AAe?$AA?5?$AAA?$AAK?$AA5?$AA7?$AA0?$AA2?$AA?5?$AAr?$AAe?$AAg?$AAi?$AAs?$AAt?$AAe?$AAr?$AA?5?$AA0?$AAx?$AA?$CF?$AAx?$AA?5?$AAf@ 100012f8     ak5702.obj
 0001:00000368       ??_C@_1CO@ENAPELKA@?$AAC?$AAA?$AAK?$AA5?$AA7?$AA0?$AA2?$AA?3?$AA?3?$AAW?$AAr?$AAi?$AAt?$AAe?$AAR?$AAe?$AAg?$AAi?$AAs?$AAt?$AAe?$AAr?$AA?$AA@ 10001368     ak5702.obj
 0001:000003e0       ??_C@_1GE@MALGICAN@?$AAS?$AAa?$AAm?$AAp?$AAl?$AAe?$AAR?$AAa?$AAt?$AAe?$AA?$DO?$AA4?$AA8?$AAK?$AA?5?$AAi?$AAs?$AA?5?$AAn?$AAo?$AAt?$AA?5?$AAs?$AAu?$AAp?$AAp?$AAo?$AAr?$AAt?$AAe?$AAd?$AA?5@ 100013e0     bsphwctxt.obj
 0001:00000448       ??_C@_1EG@HNGKJHAH@?$AAW?$AAA?$AAV?$AA_?$AAI?$AAo?$AAC?$AAo?$AAn?$AAt?$AAr?$AAo?$AAl?$AA?3?$AA?5?$AAu?$AAn?$AAt?$AAr?$AAu?$AAs?$AAt?$AAe?$AAd?$AA?5?$AAp?$AAr?$AAo?$AAc?$AAe?$AAs?$AAs@ 10001448     esai_common_topaz_v1:wavemain.obj
 0001:0000050c       ??_7InputDeviceContext@@6B@ 1000150c     esai_common_topaz_v1:hwctxt.obj
 0001:00000534       ??_7OutputDeviceContext@@6B@ 10001534     esai_common_topaz_v1:hwctxt.obj
 0001:00000560       ??_C@_1GM@MBFOFELI@?$AA?$FL?$AAE?$AAR?$AAR?$AAO?$AAR?$AA?$FN?$AA?5?$AA?$CC?$AAF?$AAa?$AAi?$AAl?$AAe?$AAd?$AA?5?$AAt?$AAo?$AA?5?$AAi?$AAn?$AAi?$AAt?$AAi?$AAa?$AAl?$AAi?$AAz?$AAe?$AA?5?$AAd?$AAi@ 10001560     esai_common_topaz_v1:hwctxt.obj
 0001:000005d0       ??_C@_1HC@FLCGCADO@?$AA?$FL?$AAE?$AAR?$AAR?$AAO?$AAR?$AA?$FN?$AA?5?$AA?$CC?$AAF?$AAa?$AAi?$AAl?$AAe?$AAd?$AA?5?$AAt?$AAo?$AA?5?$AAi?$AAn?$AAi?$AAt?$AAi?$AAa?$AAl?$AAi?$AAz?$AAe?$AA?5?$AAo?$AAu@ 100015d0     esai_common_topaz_v1:hwctxt.obj
 0001:00000648       ??_C@_1FE@JMDKDDKE@?$AA?$FL?$AAE?$AAR?$AAR?$AAO?$AAR?$AA?$FN?$AA?5?$AA?$CC?$AAI?$AAn?$AAi?$AAt?$AAi?$AAa?$AAl?$AAi?$AAz?$AAe?$AA?5?$AAA?$AAu?$AAd?$AAi?$AAo?$AA?5?$AAC?$AAo?$AAd?$AAe?$AAc?$AA?5@ 10001648     esai_common_topaz_v1:hwctxt.obj
 0001:000006a0       ??_C@_1FC@JDBMDICJ@?$AA?$FL?$AAE?$AAR?$AAR?$AAO?$AAR?$AA?$FN?$AA?5?$AA?$CC?$AAM?$AAm?$AAM?$AAa?$AAp?$AAI?$AAo?$AAS?$AAp?$AAa?$AAc?$AAe?$AA?5?$AAf?$AAa?$AAi?$AAl?$AAe?$AAd?$AA?5?$AAf?$AAo?$AAr@ 100016a0     esai_common_topaz_v1:hwctxt.obj
 0001:000006f8       ??_C@_1GE@JLPKGJBM@?$AA?$FL?$AAE?$AAR?$AAR?$AAO?$AAR?$AA?$FN?$AA?5?$AA?$CC?$AAI?$AAn?$AAi?$AAt?$AAO?$AAu?$AAt?$AAp?$AAu?$AAt?$AAD?$AAM?$AAA?$AA?3?$AA?5?$AAS?$AAy?$AAs?$AAi?$AAn?$AAt?$AAr?$AA?5@ 100016f8     esai_common_topaz_v1:hwctxt.obj
 0001:00000760       ??_C@_1GI@DIOKBAMH@?$AA?$FL?$AAE?$AAR?$AAR?$AAO?$AAR?$AA?$FN?$AA?5?$AA?$CC?$AAI?$AAn?$AAi?$AAt?$AAO?$AAu?$AAt?$AAp?$AAu?$AAt?$AAD?$AAM?$AAA?$AA?3?$AA?5?$AAD?$AAD?$AAK?$AAS?$AAd?$AAm?$AAa?$AAA@ 10001760     esai_common_topaz_v1:hwctxt.obj
 0001:000007c8       ??_C@_1GE@CGBHHGFP@?$AA?$FL?$AAE?$AAR?$AAR?$AAO?$AAR?$AA?$FN?$AA?5?$AA?$CC?$AAI?$AAn?$AAi?$AAt?$AAO?$AAu?$AAt?$AAp?$AAu?$AAt?$AAD?$AAM?$AAA?$AA?3?$AA?5?$AAD?$AAD?$AAK?$AAS?$AAd?$AAm?$AAa?$AAO@ 100017c8     esai_common_topaz_v1:hwctxt.obj
 0001:00000830       ??_C@_1HK@EHPEHBIH@?$AA?$FL?$AAE?$AAR?$AAR?$AAO?$AAR?$AA?$FN?$AA?5?$AA?$CC?$AAI?$AAn?$AAi?$AAt?$AAO?$AAu?$AAt?$AAp?$AAu?$AAt?$AAD?$AAM?$AAA?$AA?3?$AA?5?$AAD?$AAM?$AAA?$AA?5?$AAb?$AAu?$AAf?$AAf@ 10001830     esai_common_topaz_v1:hwctxt.obj
 0001:000008b0       ??_C@_1HK@PBBJOECN@?$AA?$FL?$AAE?$AAR?$AAR?$AAO?$AAR?$AA?$FN?$AA?5?$AA?$CC?$AAI?$AAn?$AAi?$AAt?$AAO?$AAu?$AAt?$AAp?$AAu?$AAt?$AAD?$AAM?$AAA?$AA?3?$AA?5?$AAB?$AAU?$AAF?$AAF?$AAE?$AAR?$AA_?$AAB@ 100018b0     esai_common_topaz_v1:hwctxt.obj
 0001:00000930       ??_C@_1HK@HFBMHBPN@?$AA?$FL?$AAE?$AAR?$AAR?$AAO?$AAR?$AA?$FN?$AA?5?$AA?$CC?$AAI?$AAn?$AAi?$AAt?$AAO?$AAu?$AAt?$AAp?$AAu?$AAt?$AAD?$AAM?$AAA?$AA?3?$AA?5?$AAB?$AAU?$AAF?$AAF?$AAE?$AAR?$AA_?$AAA@ 10001930     esai_common_topaz_v1:hwctxt.obj
 0001:000009b0       ??_C@_1FO@LLNJHCHH@?$AA?$FL?$AAE?$AAR?$AAR?$AAO?$AAR?$AA?$FN?$AA?5?$AA?$CC?$AAI?$AAn?$AAi?$AAt?$AAO?$AAu?$AAt?$AAp?$AAu?$AAt?$AAD?$AAM?$AAA?$AA?3?$AA?5?$AAI?$AAn?$AAv?$AAa?$AAl?$AAi?$AAd?$AA?5@ 100019b0     esai_common_topaz_v1:hwctxt.obj
 0001:00000a10       ??_C@_1GC@OFELANKM@?$AA?$FL?$AAE?$AAR?$AAR?$AAO?$AAR?$AA?$FN?$AA?5?$AA?$CC?$AAI?$AAn?$AAi?$AAt?$AAI?$AAn?$AAp?$AAu?$AAt?$AAD?$AAM?$AAA?$AA?3?$AA?5?$AAS?$AAy?$AAs?$AAi?$AAn?$AAt?$AAr?$AA?5?$AAr@ 10001a10     esai_common_topaz_v1:hwctxt.obj
 0001:00000a78       ??_C@_1GG@CACFPOGD@?$AA?$FL?$AAE?$AAR?$AAR?$AAO?$AAR?$AA?$FN?$AA?5?$AA?$CC?$AAI?$AAn?$AAi?$AAt?$AAI?$AAn?$AAp?$AAu?$AAt?$AAD?$AAM?$AAA?$AA?3?$AA?5?$AAD?$AAD?$AAK?$AAS?$AAd?$AAm?$AAa?$AAA?$AAl@ 10001a78     esai_common_topaz_v1:hwctxt.obj
 0001:00000ae0       ??_C@_1GC@FIKGBCOP@?$AA?$FL?$AAE?$AAR?$AAR?$AAO?$AAR?$AA?$FN?$AA?5?$AA?$CC?$AAI?$AAn?$AAi?$AAt?$AAI?$AAn?$AAp?$AAu?$AAt?$AAD?$AAM?$AAA?$AA?3?$AA?5?$AAD?$AAD?$AAK?$AAS?$AAd?$AAm?$AAa?$AAO?$AAp@ 10001ae0     esai_common_topaz_v1:hwctxt.obj
 0001:00000b48       ??_C@_1HI@EALOLDLM@?$AA?$FL?$AAE?$AAR?$AAR?$AAO?$AAR?$AA?$FN?$AA?5?$AA?$CC?$AAI?$AAn?$AAi?$AAt?$AAI?$AAn?$AAp?$AAu?$AAt?$AAD?$AAM?$AAA?$AA?3?$AA?5?$AAD?$AAM?$AAA?$AA?5?$AAb?$AAu?$AAf?$AAf?$AAe@ 10001b48     esai_common_topaz_v1:hwctxt.obj
 0001:00000bc0       ??_C@_1HI@PGFDCGBG@?$AA?$FL?$AAE?$AAR?$AAR?$AAO?$AAR?$AA?$FN?$AA?5?$AA?$CC?$AAI?$AAn?$AAi?$AAt?$AAI?$AAn?$AAp?$AAu?$AAt?$AAD?$AAM?$AAA?$AA?3?$AA?5?$AAB?$AAU?$AAF?$AAF?$AAE?$AAR?$AA_?$AAB?$AA?5@ 10001bc0     esai_common_topaz_v1:hwctxt.obj
 0001:00000c38       ??_C@_1HI@HCFGLDMG@?$AA?$FL?$AAE?$AAR?$AAR?$AAO?$AAR?$AA?$FN?$AA?5?$AA?$CC?$AAI?$AAn?$AAi?$AAt?$AAI?$AAn?$AAp?$AAu?$AAt?$AAD?$AAM?$AAA?$AA?3?$AA?5?$AAB?$AAU?$AAF?$AAF?$AAE?$AAR?$AA_?$AAA?$AA?5@ 10001c38     esai_common_topaz_v1:hwctxt.obj
 0001:00000cb0       ??_C@_1FM@OIAIFOP@?$AA?$FL?$AAE?$AAR?$AAR?$AAO?$AAR?$AA?$FN?$AA?5?$AA?$CC?$AAI?$AAn?$AAi?$AAt?$AAI?$AAn?$AAp?$AAu?$AAt?$AAD?$AAM?$AAA?$AA?3?$AA?5?$AAI?$AAn?$AAv?$AAa?$AAl?$AAi?$AAd?$AA?5?$AAs@ 10001cb0     esai_common_topaz_v1:hwctxt.obj
 0001:00000d0c       ??_C@_1BI@BHLBGEOK@?$AAP?$AAr?$AAi?$AAo?$AAr?$AAi?$AAt?$AAy?$AA2?$AA5?$AA6?$AA?$AA@ 10001d0c     esai_common_topaz_v1:hwctxt.obj
 0001:00000d28       ??_C@_1KK@JEOCOOEC@?$AA?$FL?$AAE?$AAR?$AAR?$AAO?$AAR?$AA?$FN?$AA?5?$AA?$CC?$AAU?$AAn?$AAa?$AAb?$AAl?$AAe?$AA?5?$AAt?$AAo?$AA?5?$AAc?$AAr?$AAe?$AAa?$AAt?$AAe?$AA?5?$AAa?$AAu?$AAd?$AAi?$AAo?$AA?5@ 10001d28     esai_common_topaz_v1:hwctxt.obj
 0001:00000dd8       ??_C@_1FE@OGEABEJC@?$AA?$FL?$AAE?$AAR?$AAR?$AAO?$AAR?$AA?$FN?$AA?5?$AA?$CC?$AAU?$AAn?$AAa?$AAb?$AAl?$AAe?$AA?5?$AAt?$AAo?$AA?5?$AAc?$AAr?$AAe?$AAa?$AAt?$AAe?$AA?5?$AAd?$AAe?$AAl?$AAa?$AAy?$AA?5@ 10001dd8     esai_common_topaz_v1:hwctxt.obj
 0001:00000e30       ??_C@_1JA@KMMGDDKB@?$AA?$FL?$AAE?$AAR?$AAR?$AAO?$AAR?$AA?$FN?$AA?5?$AA?$CC?$AAS?$AAt?$AAa?$AAr?$AAt?$AAO?$AAu?$AAt?$AAp?$AAu?$AAt?$AAD?$AAM?$AAA?$AA?3?$AA?5?$AAU?$AAn?$AAa?$AAb?$AAl?$AAe?$AA?5@ 10001e30     esai_common_topaz_v1:hwctxt.obj
 0001:00000ec0       ??_C@_1IO@PIJKJFCE@?$AA?$FL?$AAE?$AAR?$AAR?$AAO?$AAR?$AA?$FN?$AA?5?$AA?$CC?$AAS?$AAt?$AAa?$AAr?$AAt?$AAI?$AAn?$AAp?$AAu?$AAt?$AAD?$AAM?$AAA?$AA?3?$AA?5?$AAU?$AAn?$AAa?$AAb?$AAl?$AAe?$AA?5?$AAt@ 10001ec0     esai_common_topaz_v1:hwctxt.obj
 0001:00000f50       ??_C@_1IC@JIBANBOM@?$AAS?$AAt?$AAa?$AAr?$AAt?$AAI?$AAn?$AAp?$AAu?$AAt?$AAD?$AAM?$AAA?$AA?3?$AA?5?$AAR?$AAe?$AAc?$AAo?$AAr?$AAd?$AAi?$AAn?$AAg?$AA?5?$AAc?$AAa?$AAn?$AA?5?$AAn?$AAo?$AAt@ 10001f50     esai_common_topaz_v1:hwctxt.obj
 0001:00000fd8       ??_C@_1HC@IDPKCCMA@?$AA?$FL?$AAE?$AAR?$AAR?$AAO?$AAR?$AA?$FN?$AA?5?$AA?$CC?$AAE?$AAr?$AAr?$AAo?$AAr?$AA?5?$AAf?$AAl?$AAa?$AAg?$AA?5?$AAs?$AAe?$AAt?$AA?5?$AAi?$AAn?$AA?5?$AAo?$AAu?$AAt?$AAp?$AAu@ 10001fd8     esai_common_topaz_v1:hwctxt.obj
 0001:00001050       ??_C@_1HC@EKOFCKHP@?$AA?$FL?$AAE?$AAR?$AAR?$AAO?$AAR?$AA?$FN?$AA?5?$AA?$CC?$AAE?$AAr?$AAr?$AAo?$AAr?$AA?5?$AAf?$AAl?$AAa?$AAg?$AA?5?$AAs?$AAe?$AAt?$AA?5?$AAi?$AAn?$AA?5?$AAo?$AAu?$AAt?$AAp?$AAu@ 10002050     esai_common_topaz_v1:hwctxt.obj
 0001:000010c8       ??_C@_1GI@JJHJOGE@?$AA?$FL?$AAE?$AAR?$AAR?$AAO?$AAR?$AA?$FN?$AA?5?$AA?$CC?$AAC?$AAo?$AAu?$AAl?$AAd?$AA?5?$AAn?$AAo?$AAt?$AA?5?$AAr?$AAe?$AAt?$AAr?$AAi?$AAe?$AAv?$AAe?$AA?5?$AAo?$AAu?$AAt?$AAp@ 100020c8     esai_common_topaz_v1:hwctxt.obj
 0001:00001130       ??_C@_1FK@LCONGMCG@?$AA?$FL?$AAE?$AAR?$AAR?$AAO?$AAR?$AA?$FN?$AA?5?$AA?$CC?$AAE?$AAr?$AAr?$AAo?$AAr?$AA?5?$AAf?$AAl?$AAa?$AAg?$AA?5?$AAs?$AAe?$AAt?$AA?5?$AAi?$AAn?$AA?5?$AAi?$AAn?$AAp?$AAu?$AAt@ 10002130     esai_common_topaz_v1:hwctxt.obj
 0001:00001190       ??_C@_1HA@NFNHLKKL@?$AA?$FL?$AAE?$AAR?$AAR?$AAO?$AAR?$AA?$FN?$AA?5?$AA?$CC?$AAE?$AAr?$AAr?$AAo?$AAr?$AA?5?$AAf?$AAl?$AAa?$AAg?$AA?5?$AAs?$AAe?$AAt?$AA?5?$AAi?$AAn?$AA?5?$AAi?$AAn?$AAp?$AAu?$AAt@ 10002190     esai_common_topaz_v1:hwctxt.obj
 0001:00001200       ??_C@_1GG@LDFKJMLF@?$AA?$FL?$AAE?$AAR?$AAR?$AAO?$AAR?$AA?$FN?$AA?5?$AA?$CC?$AAC?$AAo?$AAu?$AAl?$AAd?$AA?5?$AAn?$AAo?$AAt?$AA?5?$AAr?$AAe?$AAt?$AAr?$AAi?$AAe?$AAv?$AAe?$AA?5?$AAi?$AAn?$AAp?$AAu@ 10002200     esai_common_topaz_v1:hwctxt.obj
 0001:00001268       ??_C@_1DC@CBAPFGDJ@?$AAS?$AAk?$AAi?$AAp?$AA?5?$AAd?$AAi?$AAs?$AAa?$AAb?$AAl?$AAi?$AAn?$AAg?$AA?5?$AAt?$AAh?$AAe?$AA?5?$AAA?$AAD?$AAC?$AA?$AN?$AA?6?$AA?$AA@ 10002268     esai_common_topaz_v1:hwctxt.obj
 0001:0000129c       ??_C@_1DC@FPIFOKGN@?$AAS?$AAk?$AAi?$AAp?$AA?5?$AAd?$AAi?$AAs?$AAa?$AAb?$AAl?$AAi?$AAn?$AAg?$AA?5?$AAt?$AAh?$AAe?$AA?5?$AAD?$AAA?$AAC?$AA?$AN?$AA?6?$AA?$AA@ 1000229c     esai_common_topaz_v1:hwctxt.obj
 0001:000012d0       ??_C@_1DA@JGEIEGNJ@?$AAo?$AAp?$AAe?$AAn?$AA?5?$AAa?$AAs?$AAr?$AAc?$AA?5?$AAp?$AAa?$AAi?$AAr?$AA?5?$AAf?$AAa?$AAi?$AAl?$AAe?$AAd?$AA?$AN?$AA?6?$AA?$AA@ 100022d0     esai_common_topaz_v1:hwctxt.obj
 0001:00001300       ??_7DeviceContext@@6B@     10002300     esai_common_topaz_v1:devctxt.obj
 0001:000013f0       ??_7InputStreamContextEx@@6B@ 100023f0     esai_common_topaz_v1:devctxt.obj
 0001:00001438       ??_7InputStreamContext@@6B@ 10002438     esai_common_topaz_v1:devctxt.obj
 0001:00001480       ??_7WaveStreamContext@@6B@ 10002480     esai_common_topaz_v1:devctxt.obj
 0001:000014c8       ??_7OutputStreamContextEx@@6B@ 100024c8     esai_common_topaz_v1:devctxt.obj
 0001:00001510       ??_7OutputStreamContextM8@@6B@ 10002510     esai_common_topaz_v1:devctxt.obj
 0001:00001558       ??_7OutputStreamContextS8@@6B@ 10002558     esai_common_topaz_v1:devctxt.obj
 0001:000015a0       ??_7OutputStreamContextM16@@6B@ 100025a0     esai_common_topaz_v1:devctxt.obj
 0001:000015e8       ??_7OutputStreamContextS16@@6B@ 100025e8     esai_common_topaz_v1:devctxt.obj
 0001:00001630       ??_7OutputStreamContext@@6B@ 10002630     esai_common_topaz_v1:devctxt.obj
 0001:00001818       ??_7StreamContext@@6B@     10002818     esai_common_topaz_v1:strmctxt.obj
 0001:00001858       ??_C@_1GI@EBFCCJC@?$AAE?$AAX?$AAC?$AAE?$AAP?$AAT?$AAI?$AAO?$AAN?$AA?5?$AAI?$AAN?$AA?5?$AAI?$AAS?$AAT?$AA?5?$AAf?$AAo?$AAr?$AA?5?$AAs?$AAt?$AAr?$AAe?$AAa?$AAm?$AA?5?$AA0?$AAx?$AA?$CF?$AAx@ 10002858     esai_common_topaz_v1:strmctxt.obj
 0001:000018c0       ??_C@_1BC@JBIMOOCB@?$AAP?$AAl?$AAa?$AAy?$AAb?$AAa?$AAc?$AAk?$AA?$AA@ 100028c0     esai_common_topaz_v1:mixerdrv.obj
 0001:000018d4       ??_C@_1BA@EEOGCIBB@?$AAL?$AAi?$AAn?$AAe?$AA?5?$AAI?$AAn?$AA?$AA@ 100028d4     esai_common_topaz_v1:mixerdrv.obj
 0001:000018e4       ??_C@_1BG@OGJPAHBK@?$AAM?$AAi?$AAc?$AAr?$AAo?$AAp?$AAh?$AAo?$AAn?$AAe?$AA?$AA@ 100028e4     esai_common_topaz_v1:mixerdrv.obj
 0001:000018fc       ??_C@_1CE@BJPEGCKG@?$AAR?$AAe?$AAc?$AAo?$AAr?$AAd?$AAi?$AAn?$AAg?$AA?5?$AAC?$AAo?$AAn?$AAt?$AAr?$AAo?$AAl?$AA?$AA@ 100028fc     esai_common_topaz_v1:mixerdrv.obj
 0001:00001920       ??_C@_1CA@KOFAABPH@?$AAR?$AAe?$AAc?$AAo?$AAr?$AAd?$AAi?$AAn?$AAg?$AA?5?$AAC?$AAo?$AAn?$AAt?$AAr?$AA?$AA@ 10002920     esai_common_topaz_v1:mixerdrv.obj
 0001:00001940       ??_C@_1CC@OALPFLIM@?$AAP?$AAl?$AAa?$AAy?$AAb?$AAa?$AAc?$AAk?$AA?5?$AAC?$AAo?$AAn?$AAt?$AAr?$AAo?$AAl?$AA?$AA@ 10002940     esai_common_topaz_v1:mixerdrv.obj
 0001:00001964       ??_C@_1BO@OJJBHHKI@?$AAP?$AAl?$AAa?$AAy?$AAb?$AAa?$AAc?$AAk?$AA?5?$AAC?$AAo?$AAn?$AAt?$AAr?$AA?$AA@ 10002964     esai_common_topaz_v1:mixerdrv.obj
 0001:00001988       ??_C@_1EG@GKAFBHEE@?$AAM?$AAI?$AAX?$AAE?$AAR?$AAC?$AAO?$AAN?$AAT?$AAR?$AAO?$AAL?$AA_?$AAC?$AAO?$AAN?$AAT?$AAR?$AAO?$AAL?$AAT?$AAY?$AAP?$AAE?$AA_?$AAM?$AAI?$AAL?$AAL?$AAI?$AAT?$AAI@ 10002988     esai_common_topaz_v1:mixerdrv.obj
 0001:000019d0       ??_C@_1EG@KGPLLMHC@?$AAM?$AAI?$AAX?$AAE?$AAR?$AAC?$AAO?$AAN?$AAT?$AAR?$AAO?$AAL?$AA_?$AAC?$AAO?$AAN?$AAT?$AAR?$AAO?$AAL?$AAT?$AAY?$AAP?$AAE?$AA_?$AAM?$AAI?$AAC?$AAR?$AAO?$AAT?$AAI@ 100029d0     esai_common_topaz_v1:mixerdrv.obj
 0001:00001a18       ??_C@_1EG@MHHEILGF@?$AAM?$AAI?$AAX?$AAE?$AAR?$AAC?$AAO?$AAN?$AAT?$AAR?$AAO?$AAL?$AA_?$AAC?$AAO?$AAN?$AAT?$AAR?$AAO?$AAL?$AAT?$AAY?$AAP?$AAE?$AA_?$AAS?$AAT?$AAE?$AAR?$AAE?$AAO?$AAE@ 10002a18     esai_common_topaz_v1:mixerdrv.obj
 0001:00001a60       ??_C@_1DO@MOGMEDOD@?$AAM?$AAI?$AAX?$AAE?$AAR?$AAC?$AAO?$AAN?$AAT?$AAR?$AAO?$AAL?$AA_?$AAC?$AAO?$AAN?$AAT?$AAR?$AAO?$AAL?$AAT?$AAY?$AAP?$AAE?$AA_?$AAO?$AAN?$AAO?$AAF?$AAF?$AA?$AA@ 10002a60     esai_common_topaz_v1:mixerdrv.obj
 0001:00001aa0       ??_C@_1DM@DCLFABPP@?$AAM?$AAI?$AAX?$AAE?$AAR?$AAC?$AAO?$AAN?$AAT?$AAR?$AAO?$AAL?$AA_?$AAC?$AAO?$AAN?$AAT?$AAR?$AAO?$AAL?$AAT?$AAY?$AAP?$AAE?$AA_?$AAM?$AAU?$AAT?$AAE?$AA?$AA@ 10002aa0     esai_common_topaz_v1:mixerdrv.obj
 0001:00001adc       ??_C@_1DM@BCDOONIF@?$AAM?$AAI?$AAX?$AAE?$AAR?$AAC?$AAO?$AAN?$AAT?$AAR?$AAO?$AAL?$AA_?$AAC?$AAO?$AAN?$AAT?$AAR?$AAO?$AAL?$AAT?$AAY?$AAP?$AAE?$AA_?$AAM?$AAO?$AAN?$AAO?$AA?$AA@ 10002adc     esai_common_topaz_v1:mixerdrv.obj
 0001:00001b18       ??_C@_1EE@FIBKNKLH@?$AAM?$AAI?$AAX?$AAE?$AAR?$AAC?$AAO?$AAN?$AAT?$AAR?$AAO?$AAL?$AA_?$AAC?$AAO?$AAN?$AAT?$AAR?$AAO?$AAL?$AAT?$AAY?$AAP?$AAE?$AA_?$AAL?$AAO?$AAU?$AAD?$AAN?$AAE?$AAS@ 10002b18     esai_common_topaz_v1:mixerdrv.obj
 0001:00001b60       ??_C@_1EA@ONOCHFEP@?$AAM?$AAI?$AAX?$AAE?$AAR?$AAC?$AAO?$AAN?$AAT?$AAR?$AAO?$AAL?$AA_?$AAC?$AAO?$AAN?$AAT?$AAR?$AAO?$AAL?$AAT?$AAY?$AAP?$AAE?$AA_?$AAB?$AAU?$AAT?$AAT?$AAO?$AAN?$AA?$AA@ 10002b60     esai_common_topaz_v1:mixerdrv.obj
 0001:00001ba0       ??_C@_1EC@LBKFNEJB@?$AAM?$AAI?$AAX?$AAE?$AAR?$AAC?$AAO?$AAN?$AAT?$AAR?$AAO?$AAL?$AA_?$AAC?$AAO?$AAN?$AAT?$AAR?$AAO?$AAL?$AAT?$AAY?$AAP?$AAE?$AA_?$AAB?$AAO?$AAO?$AAL?$AAE?$AAA?$AAN@ 10002ba0     esai_common_topaz_v1:mixerdrv.obj
 0001:00001be8       ??_C@_1EA@JCFBIPAK@?$AAM?$AAI?$AAX?$AAE?$AAR?$AAC?$AAO?$AAN?$AAT?$AAR?$AAO?$AAL?$AA_?$AAC?$AAO?$AAN?$AAT?$AAR?$AAO?$AAL?$AAT?$AAY?$AAP?$AAE?$AA_?$AAS?$AAL?$AAI?$AAD?$AAE?$AAR?$AA?$AA@ 10002be8     esai_common_topaz_v1:mixerdrv.obj
 0001:00001c28       ??_C@_1EG@BEPOGKNO@?$AAM?$AAI?$AAX?$AAE?$AAR?$AAC?$AAO?$AAN?$AAT?$AAR?$AAO?$AAL?$AA_?$AAC?$AAO?$AAN?$AAT?$AAR?$AAO?$AAL?$AAT?$AAY?$AAP?$AAE?$AA_?$AAQ?$AAS?$AAO?$AAU?$AAN?$AAD?$AAP@ 10002c28     esai_common_topaz_v1:mixerdrv.obj
 0001:00001c70       ??_C@_1DK@HNKLKPNJ@?$AAM?$AAI?$AAX?$AAE?$AAR?$AAC?$AAO?$AAN?$AAT?$AAR?$AAO?$AAL?$AA_?$AAC?$AAO?$AAN?$AAT?$AAR?$AAO?$AAL?$AAT?$AAY?$AAP?$AAE?$AA_?$AAP?$AAA?$AAN?$AA?$AA@ 10002c70     esai_common_topaz_v1:mixerdrv.obj
 0001:00001cb0       ??_C@_1EE@PPIBPMLH@?$AAM?$AAI?$AAX?$AAE?$AAR?$AAC?$AAO?$AAN?$AAT?$AAR?$AAO?$AAL?$AA_?$AAC?$AAO?$AAN?$AAT?$AAR?$AAO?$AAL?$AAT?$AAY?$AAP?$AAE?$AA_?$AAU?$AAN?$AAS?$AAI?$AAG?$AAN?$AAE@ 10002cb0     esai_common_topaz_v1:mixerdrv.obj
 0001:00001cf8       ??_C@_1EA@PAIJNMCC@?$AAM?$AAI?$AAX?$AAE?$AAR?$AAC?$AAO?$AAN?$AAT?$AAR?$AAO?$AAL?$AA_?$AAC?$AAO?$AAN?$AAT?$AAR?$AAO?$AAL?$AAT?$AAY?$AAP?$AAE?$AA_?$AAS?$AAI?$AAG?$AAN?$AAE?$AAD?$AA?$AA@ 10002cf8     esai_common_topaz_v1:mixerdrv.obj
 0001:00001d38       ??_C@_1EC@KPFLKHEG@?$AAM?$AAI?$AAX?$AAE?$AAR?$AAC?$AAO?$AAN?$AAT?$AAR?$AAO?$AAL?$AA_?$AAC?$AAO?$AAN?$AAT?$AAR?$AAO?$AAL?$AAT?$AAY?$AAP?$AAE?$AA_?$AAP?$AAE?$AAR?$AAC?$AAE?$AAN?$AAT@ 10002d38     esai_common_topaz_v1:mixerdrv.obj
 0001:00001d80       ??_C@_1EE@FDJLOIGD@?$AAM?$AAI?$AAX?$AAE?$AAR?$AAC?$AAO?$AAN?$AAT?$AAR?$AAO?$AAL?$AA_?$AAC?$AAO?$AAN?$AAT?$AAR?$AAO?$AAL?$AAT?$AAY?$AAP?$AAE?$AA_?$AAD?$AAE?$AAC?$AAI?$AAB?$AAE?$AAL@ 10002d80     esai_common_topaz_v1:mixerdrv.obj
 0001:00001dc8       ??_C@_1EO@CIONLEIK@?$AAM?$AAI?$AAX?$AAE?$AAR?$AAC?$AAO?$AAN?$AAT?$AAR?$AAO?$AAL?$AA_?$AAC?$AAO?$AAN?$AAT?$AAR?$AAO?$AAL?$AAT?$AAY?$AAP?$AAE?$AA_?$AAU?$AAN?$AAS?$AAI?$AAG?$AAN?$AAE@ 10002dc8     esai_common_topaz_v1:mixerdrv.obj
 0001:00001e18       ??_C@_1EK@KIDDBONI@?$AAM?$AAI?$AAX?$AAE?$AAR?$AAC?$AAO?$AAN?$AAT?$AAR?$AAO?$AAL?$AA_?$AAC?$AAO?$AAN?$AAT?$AAR?$AAO?$AAL?$AAT?$AAY?$AAP?$AAE?$AA_?$AAS?$AAI?$AAG?$AAN?$AAE?$AAD?$AAM@ 10002e18     esai_common_topaz_v1:mixerdrv.obj
 0001:00001e68       ??_C@_1EG@EBKFDDEH@?$AAM?$AAI?$AAX?$AAE?$AAR?$AAC?$AAO?$AAN?$AAT?$AAR?$AAO?$AAL?$AA_?$AAC?$AAO?$AAN?$AAT?$AAR?$AAO?$AAL?$AAT?$AAY?$AAP?$AAE?$AA_?$AAP?$AAE?$AAA?$AAK?$AAM?$AAE?$AAT@ 10002e68     esai_common_topaz_v1:mixerdrv.obj
 0001:00001eb0       ??_C@_1EM@DKIPIFCO@?$AAM?$AAI?$AAX?$AAE?$AAR?$AAC?$AAO?$AAN?$AAT?$AAR?$AAO?$AAL?$AA_?$AAC?$AAO?$AAN?$AAT?$AAR?$AAO?$AAL?$AAT?$AAY?$AAP?$AAE?$AA_?$AAB?$AAO?$AAO?$AAL?$AAE?$AAA?$AAN@ 10002eb0     esai_common_topaz_v1:mixerdrv.obj
 0001:00001f00       ??_C@_1EM@KGOHBNDE@?$AAM?$AAI?$AAX?$AAE?$AAR?$AAC?$AAO?$AAN?$AAT?$AAR?$AAO?$AAL?$AA_?$AAC?$AAO?$AAN?$AAT?$AAR?$AAO?$AAL?$AAT?$AAY?$AAP?$AAE?$AA_?$AAS?$AAI?$AAN?$AAG?$AAL?$AAE?$AAS@ 10002f00     esai_common_topaz_v1:mixerdrv.obj
 0001:00001f4c       ??_C@_1DK@HHCAMDON@?$AAM?$AAI?$AAX?$AAE?$AAR?$AAC?$AAO?$AAN?$AAT?$AAR?$AAO?$AAL?$AA_?$AAC?$AAO?$AAN?$AAT?$AAR?$AAO?$AAL?$AAT?$AAY?$AAP?$AAE?$AA_?$AAM?$AAU?$AAX?$AA?$AA@ 10002f4c     esai_common_topaz_v1:mixerdrv.obj
 0001:00001f88       ??_C@_1FA@ECHLHCDJ@?$AAM?$AAI?$AAX?$AAE?$AAR?$AAC?$AAO?$AAN?$AAT?$AAR?$AAO?$AAL?$AA_?$AAC?$AAO?$AAN?$AAT?$AAR?$AAO?$AAL?$AAT?$AAY?$AAP?$AAE?$AA_?$AAM?$AAU?$AAL?$AAT?$AAI?$AAP?$AAL@ 10002f88     esai_common_topaz_v1:mixerdrv.obj
 0001:00001fd8       ??_C@_1DO@OPBKEMFB@?$AAM?$AAI?$AAX?$AAE?$AAR?$AAC?$AAO?$AAN?$AAT?$AAR?$AAO?$AAL?$AA_?$AAC?$AAO?$AAN?$AAT?$AAR?$AAO?$AAL?$AAT?$AAY?$AAP?$AAE?$AA_?$AAM?$AAI?$AAX?$AAE?$AAR?$AA?$AA@ 10002fd8     esai_common_topaz_v1:mixerdrv.obj
 0001:00002018       ??_C@_1EA@BGMJCECN@?$AAM?$AAI?$AAX?$AAE?$AAR?$AAC?$AAO?$AAN?$AAT?$AAR?$AAO?$AAL?$AA_?$AAC?$AAO?$AAN?$AAT?$AAR?$AAO?$AAL?$AAT?$AAY?$AAP?$AAE?$AA_?$AAV?$AAO?$AAL?$AAU?$AAM?$AAE?$AA?$AA@ 10003018     esai_common_topaz_v1:mixerdrv.obj
 0001:00002058       ??_C@_1EA@CECHMMMP@?$AAM?$AAI?$AAX?$AAE?$AAR?$AAC?$AAO?$AAN?$AAT?$AAR?$AAO?$AAL?$AA_?$AAC?$AAO?$AAN?$AAT?$AAR?$AAO?$AAL?$AAT?$AAY?$AAP?$AAE?$AA_?$AAT?$AAR?$AAE?$AAB?$AAL?$AAE?$AA?$AA@ 10003058     esai_common_topaz_v1:mixerdrv.obj
 0001:00002098       ??_C@_1DO@KGELIMMP@?$AAM?$AAI?$AAX?$AAE?$AAR?$AAC?$AAO?$AAN?$AAT?$AAR?$AAO?$AAL?$AA_?$AAC?$AAO?$AAN?$AAT?$AAR?$AAO?$AAL?$AAT?$AAY?$AAP?$AAE?$AA_?$AAF?$AAA?$AAD?$AAE?$AAR?$AA?$AA@ 10003098     esai_common_topaz_v1:mixerdrv.obj
 0001:000020d8       ??_C@_1EG@NLNANFDC@?$AAM?$AAI?$AAX?$AAE?$AAR?$AAC?$AAO?$AAN?$AAT?$AAR?$AAO?$AAL?$AA_?$AAC?$AAO?$AAN?$AAT?$AAR?$AAO?$AAL?$AAT?$AAY?$AAP?$AAE?$AA_?$AAE?$AAQ?$AAU?$AAA?$AAL?$AAI?$AAZ@ 100030d8     esai_common_topaz_v1:mixerdrv.obj
 0001:00002120       ??_C@_1DM@FDDIFNFI@?$AAM?$AAI?$AAX?$AAE?$AAR?$AAC?$AAO?$AAN?$AAT?$AAR?$AAO?$AAL?$AA_?$AAC?$AAO?$AAN?$AAT?$AAR?$AAO?$AAL?$AAT?$AAY?$AAP?$AAE?$AA_?$AAB?$AAA?$AAS?$AAS?$AA?$AA@ 10003120     esai_common_topaz_v1:mixerdrv.obj
 0001:00002160       ??_C@_1EA@IAIECAKO@?$AAM?$AAI?$AAX?$AAE?$AAR?$AAC?$AAO?$AAN?$AAT?$AAR?$AAO?$AAL?$AA_?$AAC?$AAO?$AAN?$AAT?$AAR?$AAO?$AAL?$AAT?$AAY?$AAP?$AAE?$AA_?$AAC?$AAU?$AAS?$AAT?$AAO?$AAM?$AA?$AA@ 10003160     esai_common_topaz_v1:mixerdrv.obj
 0001:0000225c       ?m_cControls@MixerControlList@@0KB 1000325c     esai_common_topaz_v1:mixerdrv.obj
 0001:00002260       ??_C@_1BE@ELICABCK@?$AA?$DM?$AAu?$AAn?$AAk?$AAn?$AAo?$AAw?$AAn?$AA?$DO?$AA?$AA@ 10003260     esai_common_topaz_v1:mixerdrv.obj
 0001:00002274       ??_C@_1CI@HHNFIEHC@?$AAM?$AAi?$AAx?$AAe?$AAr?$AAC?$AAa?$AAl?$AAl?$AAb?$AAa?$AAc?$AAk?$AA?$CI?$AA?$CF?$AAd?$AA?$CJ?$AA?$AN?$AA?6?$AA?$AA@ 10003274     esai_common_topaz_v1:mixerdrv.obj
 0001:0000229c       ??_C@_1BI@DKACBKCL@?$AAA?$AAu?$AAd?$AAi?$AAo?$AA?5?$AAM?$AAi?$AAx?$AAe?$AAr?$AA?$AA@ 1000329c     esai_common_topaz_v1:mixerdrv.obj
 0001:000022b8       ??_C@_1FE@BDJOHFBK@?$AA?$FL?$AAE?$AAR?$AAR?$AAO?$AAR?$AA?$FN?$AA?5?$AA?$CC?$AAw?$AAd?$AAe?$AAv?$AA_?$AAM?$AAX?$AAD?$AAM?$AA_?$AAO?$AAP?$AAE?$AAN?$AA?3?$AA?5?$AAo?$AAu?$AAt?$AA?5?$AAo?$AAf?$AA?5@ 100032b8     esai_common_topaz_v1:mixerdrv.obj
 0001:0000230c       ??_C@_1DM@CHMELAAB@?$AAG?$AAe?$AAt?$AAM?$AAi?$AAx?$AAe?$AAr?$AAL?$AAi?$AAn?$AAe?$AAI?$AAn?$AAf?$AAo?$AA?3?$AA?5?$AA?$CC?$AA?$CF?$AAs?$AA?$CC?$AA?5?$AA?$CF?$AA0?$AA8?$AAx?$AA?$AN?$AA?6?$AA?$AA@ 1000330c     esai_common_topaz_v1:mixerdrv.obj
 0001:00002348       ??_C@_1FC@LHNBJHH@?$AAG?$AAe?$AAt?$AAM?$AAi?$AAx?$AAe?$AAr?$AAL?$AAi?$AAn?$AAe?$AAI?$AAn?$AAf?$AAo?$AA?3?$AA?5?$AAi?$AAn?$AAv?$AAa?$AAl?$AAi?$AAd?$AA?5?$AAl?$AAi?$AAn?$AAe?$AA?5?$AAI@ 10003348     esai_common_topaz_v1:mixerdrv.obj
 0001:000023a0       ??_C@_1GA@DDKINBEJ@?$AAG?$AAe?$AAt?$AAM?$AAi?$AAx?$AAe?$AAr?$AAL?$AAi?$AAn?$AAe?$AAI?$AAn?$AAf?$AAo?$AA?3?$AA?5?$AAn?$AAo?$AA?5?$AAl?$AAi?$AAn?$AAe?$AA?5?$AAo?$AAf?$AA?5?$AAt?$AAa?$AAr@ 100033a0     esai_common_topaz_v1:mixerdrv.obj
 0001:00002400       ??_C@_1GG@MELCAJPL@?$AAG?$AAe?$AAt?$AAM?$AAi?$AAx?$AAe?$AAr?$AAL?$AAi?$AAn?$AAe?$AAI?$AAn?$AAf?$AAo?$AA?3?$AA?5?$AAn?$AAo?$AA?5?$AAl?$AAi?$AAn?$AAe?$AA?5?$AAo?$AAf?$AA?5?$AAc?$AAo?$AAm@ 10003400     esai_common_topaz_v1:mixerdrv.obj
 0001:00002468       ??_C@_1EO@HDKNAFNG@?$AAG?$AAe?$AAt?$AAM?$AAi?$AAx?$AAe?$AAr?$AAL?$AAi?$AAn?$AAe?$AAI?$AAn?$AAf?$AAo?$AA?3?$AA?5?$AAi?$AAn?$AAv?$AAa?$AAl?$AAi?$AAd?$AA?5?$AAq?$AAu?$AAe?$AAr?$AAy?$AA?5@ 10003468     esai_common_topaz_v1:mixerdrv.obj
 0001:000024b8       ??_C@_1DE@PIKBGEIJ@?$AAG?$AAe?$AAt?$AAM?$AAi?$AAx?$AAe?$AAr?$AAL?$AAi?$AAn?$AAe?$AAI?$AAn?$AAf?$AAo?$AA?5?$AAT?$AAA?$AAR?$AAG?$AAE?$AAT?$AA?$AN?$AA?6?$AA?$AA@ 100034b8     esai_common_topaz_v1:mixerdrv.obj
 0001:000024ec       ??_C@_1DK@COFPEFKO@?$AAG?$AAe?$AAt?$AAM?$AAi?$AAx?$AAe?$AAr?$AAL?$AAi?$AAn?$AAe?$AAI?$AAn?$AAf?$AAo?$AA?5?$AAC?$AAO?$AAM?$AAP?$AAO?$AAN?$AAE?$AAN?$AAT?$AA?$AN?$AA?6?$AA?$AA@ 100034ec     esai_common_topaz_v1:mixerdrv.obj
 0001:00002528       ??_C@_1FG@LCCLAGKB@?$AAG?$AAe?$AAt?$AAM?$AAi?$AAx?$AAe?$AAr?$AAL?$AAi?$AAn?$AAe?$AAI?$AAn?$AAf?$AAo?$AA?3?$AA?5?$AAi?$AAn?$AAv?$AAa?$AAl?$AAi?$AAd?$AA?5?$AAs?$AAo?$AAu?$AAr?$AAc?$AAe@ 10003528     esai_common_topaz_v1:mixerdrv.obj
 0001:00002580       ??_C@_1HG@JHFCMAJM@?$AAG?$AAe?$AAt?$AAM?$AAi?$AAx?$AAe?$AAr?$AAL?$AAi?$AAn?$AAe?$AAI?$AAn?$AAf?$AAo?$AA?3?$AA?5?$AAi?$AAn?$AAc?$AAo?$AAn?$AAs?$AAi?$AAs?$AAt?$AAe?$AAn?$AAt?$AA?5?$AAi@ 10003580     esai_common_topaz_v1:mixerdrv.obj
 0001:000025f8       ??_C@_1EA@IAOAGGKE@?$AAG?$AAe?$AAt?$AAM?$AAi?$AAx?$AAe?$AAr?$AAL?$AAi?$AAn?$AAe?$AAI?$AAn?$AAf?$AAo?$AA?5?$AAS?$AAO?$AAU?$AAR?$AAC?$AAE?$AA?5?$AA?$CF?$AAx?$AA?5?$AA?$CF?$AAx?$AA?$AN?$AA?6?$AA?$AA@ 100035f8     esai_common_topaz_v1:mixerdrv.obj
 0001:00002638       ??_C@_1DK@GMMCEECL@?$AAG?$AAe?$AAt?$AAM?$AAi?$AAx?$AAe?$AAr?$AAL?$AAi?$AAn?$AAe?$AAI?$AAn?$AAf?$AAo?$AA?5?$AAL?$AAI?$AAN?$AAE?$AAI?$AAD?$AA?5?$AA?$CF?$AAx?$AA?$AN?$AA?6?$AA?$AA@ 10003638     esai_common_topaz_v1:mixerdrv.obj
 0001:00002678       ??_C@_1GA@BBJIEEAD@?$AAG?$AAe?$AAt?$AAM?$AAi?$AAx?$AAe?$AAr?$AAL?$AAi?$AAn?$AAe?$AAI?$AAn?$AAf?$AAo?$AA?3?$AA?5?$AAi?$AAn?$AAv?$AAa?$AAl?$AAi?$AAd?$AA?5?$AAd?$AAe?$AAs?$AAt?$AAi?$AAn@ 10003678     esai_common_topaz_v1:mixerdrv.obj
 0001:000026d8       ??_C@_1EE@DGPNNKNM@?$AAG?$AAe?$AAt?$AAM?$AAi?$AAx?$AAe?$AAr?$AAL?$AAi?$AAn?$AAe?$AAI?$AAn?$AAf?$AAo?$AA?5?$AAD?$AAE?$AAS?$AAT?$AAI?$AAN?$AAA?$AAT?$AAI?$AAO?$AAN?$AA?5?$AA?$CF?$AAx?$AA?$AN@ 100036d8     esai_common_topaz_v1:mixerdrv.obj
 0001:00002720       ??_C@_1FG@OKMEMBEL@?$AAG?$AAe?$AAt?$AAM?$AAi?$AAx?$AAe?$AAr?$AAL?$AAi?$AAn?$AAe?$AAC?$AAo?$AAn?$AAt?$AAr?$AAo?$AAl?$AAs?$AA?3?$AA?5?$AAi?$AAn?$AAv?$AAa?$AAl?$AAi?$AAd?$AA?5?$AAq?$AAu@ 10003720     esai_common_topaz_v1:mixerdrv.obj
 0001:00002778       ??_C@_1IG@OCFKLJPN@?$AAG?$AAe?$AAt?$AAM?$AAi?$AAx?$AAe?$AAr?$AAL?$AAi?$AAn?$AAe?$AAC?$AAo?$AAn?$AAt?$AAr?$AAo?$AAl?$AAs?$AA?3?$AA?5?$AAl?$AAi?$AAn?$AAe?$AA?5?$AA?$CF?$AA0?$AA4?$AAx?$AA?5@ 10003778     esai_common_topaz_v1:mixerdrv.obj
 0001:00002800       ??_C@_1GO@CMCLLJCP@?$AAG?$AAe?$AAt?$AAM?$AAi?$AAx?$AAe?$AAr?$AAL?$AAi?$AAn?$AAe?$AAC?$AAo?$AAn?$AAt?$AAr?$AAo?$AAl?$AAs?$AA?3?$AA?5?$AAc?$AAo?$AAn?$AAt?$AAr?$AAo?$AAl?$AA?5?$AAc?$AAo@ 10003800     esai_common_topaz_v1:mixerdrv.obj
 0001:00002870       ??_C@_1EM@NAGBJFBM@?$AAG?$AAe?$AAt?$AAM?$AAi?$AAx?$AAe?$AAr?$AAL?$AAi?$AAn?$AAe?$AAC?$AAo?$AAn?$AAt?$AAr?$AAo?$AAl?$AAs?$AA?3?$AA?5?$AAO?$AAN?$AAE?$AAB?$AAY?$AAT?$AAY?$AAP?$AAE?$AA?5@ 10003870     esai_common_topaz_v1:mixerdrv.obj
 0001:000028c0       ??_C@_1GM@MONMFDNB@?$AAG?$AAe?$AAt?$AAM?$AAi?$AAx?$AAe?$AAr?$AAL?$AAi?$AAn?$AAe?$AAC?$AAo?$AAn?$AAt?$AAr?$AAo?$AAl?$AAs?$AA?3?$AA?5?$AAc?$AAo?$AAn?$AAt?$AAr?$AAo?$AAl?$AA?5?$AAc?$AAo@ 100038c0     esai_common_topaz_v1:mixerdrv.obj
 0001:00002930       ??_C@_1EG@IPGPLBHF@?$AAG?$AAe?$AAt?$AAM?$AAi?$AAx?$AAe?$AAr?$AAL?$AAi?$AAn?$AAe?$AAC?$AAo?$AAn?$AAt?$AAr?$AAo?$AAl?$AAs?$AA?3?$AA?5?$AAO?$AAN?$AAE?$AAB?$AAY?$AAI?$AAD?$AA?5?$AA?$CF?$AAx@ 10003930     esai_common_topaz_v1:mixerdrv.obj
 0001:00002978       ??_C@_1JG@CANNPDPK@?$AAG?$AAe?$AAt?$AAM?$AAi?$AAx?$AAe?$AAr?$AAL?$AAi?$AAn?$AAe?$AAC?$AAo?$AAn?$AAt?$AAr?$AAo?$AAl?$AAs?$AA?3?$AA?5?$AAi?$AAn?$AAc?$AAo?$AAr?$AAr?$AAe?$AAc?$AAt?$AA?5@ 10003978     esai_common_topaz_v1:mixerdrv.obj
 0001:00002a10       ??_C@_1FK@PFCBAFBC@?$AAG?$AAe?$AAt?$AAM?$AAi?$AAx?$AAe?$AAr?$AAL?$AAi?$AAn?$AAe?$AAC?$AAo?$AAn?$AAt?$AAr?$AAo?$AAl?$AAs?$AA?3?$AA?5?$AAi?$AAn?$AAv?$AAa?$AAl?$AAi?$AAd?$AA?5?$AAl?$AAi@ 10003a10     esai_common_topaz_v1:mixerdrv.obj
 0001:00002a6c       ??_C@_1DO@KJNHEOOA@?$AAG?$AAe?$AAt?$AAM?$AAi?$AAx?$AAe?$AAr?$AAL?$AAi?$AAn?$AAe?$AAC?$AAo?$AAn?$AAt?$AAr?$AAo?$AAl?$AAs?$AA?3?$AA?5?$AAA?$AAL?$AAL?$AA?5?$AA?$CF?$AAx?$AA?$AN?$AA?6?$AA?$AA@ 10003a6c     esai_common_topaz_v1:mixerdrv.obj
 0001:00002aac       ??_C@_1DK@HNFPDNP@?$AAG?$AAe?$AAt?$AAM?$AAi?$AAx?$AAe?$AAr?$AAC?$AAo?$AAn?$AAt?$AAr?$AAo?$AAl?$AAD?$AAe?$AAt?$AAa?$AAi?$AAl?$AAs?$AA?$CI?$AA?$CF?$AAd?$AA?$CJ?$AA?$AN?$AA?6?$AA?$AA@ 10003aac     esai_common_topaz_v1:mixerdrv.obj
 0001:00002ae8       ??_C@_1DK@IAOOCHGE@?$AAS?$AAe?$AAt?$AAM?$AAi?$AAx?$AAe?$AAr?$AAC?$AAo?$AAn?$AAt?$AAr?$AAo?$AAl?$AAD?$AAe?$AAt?$AAa?$AAi?$AAl?$AAs?$AA?$CI?$AA?$CF?$AAd?$AA?$CJ?$AA?$AN?$AA?6?$AA?$AA@ 10003ae8     esai_common_topaz_v1:mixerdrv.obj
 0001:00002b24       ??_7MixerControlList@@6B@  10003b24     esai_common_topaz_v1:mixerdrv.obj
 0001:00002b28       ??_7MixerControlVolumeMaster@@6B@ 10003b28     esai_common_topaz_v1:mixerdrv.obj
 0001:00002b4c       ??_7MixerControlVolume@@6B@ 10003b4c     esai_common_topaz_v1:mixerdrv.obj
 0001:00002b70       ??_7MixerControl@@6B@      10003b70     esai_common_topaz_v1:mixerdrv.obj
 0001:00002b90       ??_C@_1GA@LNIMIIDM@?$AAS?$AAe?$AAt?$AAM?$AAi?$AAx?$AAe?$AAr?$AAC?$AAo?$AAn?$AAt?$AAr?$AAo?$AAl?$AAD?$AAe?$AAt?$AAa?$AAi?$AAl?$AAs?$AA?3?$AA?5?$AAV?$AAo?$AAl?$AAu?$AAm?$AAe?$AA?5?$AAe@ 10003b90     esai_common_topaz_v1:mixerdrv.obj
 0001:00002bf0       ??_C@_1BM@DBCMFCBE@?$AAM?$AAa?$AAs?$AAt?$AAe?$AAr?$AA?5?$AAV?$AAo?$AAl?$AAu?$AAm?$AAe?$AA?$AA@ 10003bf0     esai_common_topaz_v1:mixerdrv.obj
 0001:00002c0c       ??_7MixerControlVolumeMic@@6B@ 10003c0c     esai_common_topaz_v1:mixerdrv.obj
 0001:00002c30       ??_C@_1BG@LAGONMFD@?$AAM?$AAi?$AAc?$AA?5?$AAV?$AAo?$AAl?$AAu?$AAm?$AAe?$AA?$AA@ 10003c30     esai_common_topaz_v1:mixerdrv.obj
 0001:00002c48       ??_7MixerControlMuteMaster@@6B@ 10003c48     esai_common_topaz_v1:mixerdrv.obj
 0001:00002c6c       ??_7MixerControlBoolean@@6B@ 10003c6c     esai_common_topaz_v1:mixerdrv.obj
 0001:00002c90       ??_C@_1BI@PEAJCPFH@?$AAM?$AAa?$AAs?$AAt?$AAe?$AAr?$AA?5?$AAM?$AAu?$AAt?$AAe?$AA?$AA@ 10003c90     esai_common_topaz_v1:mixerdrv.obj
 0001:00002ca8       ??_7MixerControlMuteMic@@6B@ 10003ca8     esai_common_topaz_v1:mixerdrv.obj
 0001:00002ccc       ??_C@_1BC@MOMKCGGI@?$AAM?$AAi?$AAc?$AA?5?$AAM?$AAu?$AAt?$AAe?$AA?$AA@ 10003ccc     esai_common_topaz_v1:mixerdrv.obj
 0001:00002ce0       ??_7MixerControlLoopback@@6B@ 10003ce0     esai_common_topaz_v1:mixerdrv.obj
 0001:00002d04       ??_C@_1BC@NMCMBANA@?$AAL?$AAo?$AAo?$AAp?$AAb?$AAa?$AAc?$AAk?$AA?$AA@ 10003d04     esai_common_topaz_v1:mixerdrv.obj
 0001:00002d18       ??_C@_1CC@NMFCMAHN@?$AAL?$AAo?$AAo?$AAp?$AAb?$AAa?$AAc?$AAk?$AA?5?$AAC?$AAo?$AAn?$AAt?$AAr?$AAo?$AAl?$AA?$AA@ 10003d18     esai_common_topaz_v1:mixerdrv.obj
 0001:00002d3c       ??_7MixerControlInputMux@@6B@ 10003d3c     esai_common_topaz_v1:mixerdrv.obj
 0001:00002d58       ??_C@_1BE@FNMPOHBO@?$AAI?$AAn?$AAp?$AAu?$AAt?$AA?5?$AAM?$AAu?$AAx?$AA?$AA@ 10003d58     esai_common_topaz_v1:mixerdrv.obj
 0001:00002d70       ??_C@_1EM@DBPFHEAH@?$AA?$FL?$AAE?$AAR?$AAR?$AAO?$AAR?$AA?$FN?$AA?5?$AA?$CC?$AAU?$AAn?$AAs?$AAu?$AAp?$AAp?$AAo?$AAr?$AAt?$AAe?$AAd?$AA?5?$AAm?$AAi?$AAx?$AAe?$AAr?$AA?5?$AAm?$AAe?$AAs?$AAs?$AAa@ 10003d70     esai_common_topaz_v1:mixerdrv.obj
 0001:00002dbc       ??_C@_1DC@MEFIDC@?$AAM?$AAX?$AAD?$AAM?$AA_?$AAS?$AAE?$AAT?$AAC?$AAO?$AAN?$AAT?$AAR?$AAO?$AAL?$AAD?$AAE?$AAT?$AAA?$AAI?$AAL?$AAS?$AA?$AN?$AA?6?$AA?$AA@ 10003dbc     esai_common_topaz_v1:mixerdrv.obj
 0001:00002df0       ??_C@_1DC@CEKCBIBD@?$AAM?$AAX?$AAD?$AAM?$AA_?$AAG?$AAE?$AAT?$AAC?$AAO?$AAN?$AAT?$AAR?$AAO?$AAL?$AAD?$AAE?$AAT?$AAA?$AAI?$AAL?$AAS?$AA?$AN?$AA?6?$AA?$AA@ 10003df0     esai_common_topaz_v1:mixerdrv.obj
 0001:00002e24       ??_C@_1CO@OJFEDBFL@?$AAM?$AAX?$AAD?$AAM?$AA_?$AAG?$AAE?$AAT?$AAL?$AAI?$AAN?$AAE?$AAC?$AAO?$AAN?$AAT?$AAR?$AAO?$AAL?$AAS?$AA?$AN?$AA?6?$AA?$AA@ 10003e24     esai_common_topaz_v1:mixerdrv.obj
 0001:00002e54       ??_C@_1CG@CLPEJCBP@?$AAM?$AAX?$AAD?$AAM?$AA_?$AAG?$AAE?$AAT?$AAL?$AAI?$AAN?$AAE?$AAI?$AAN?$AAF?$AAO?$AA?$AN?$AA?6?$AA?$AA@ 10003e54     esai_common_topaz_v1:mixerdrv.obj
 0001:00002e7c       ??_C@_1BK@DOLEBCGM@?$AAM?$AAX?$AAD?$AAM?$AA_?$AAC?$AAL?$AAO?$AAS?$AAE?$AA?$AN?$AA?6?$AA?$AA@ 10003e7c     esai_common_topaz_v1:mixerdrv.obj
 0001:00002e98       ??_C@_1BI@FCEHOKDK@?$AAM?$AAX?$AAD?$AAM?$AA_?$AAO?$AAP?$AAE?$AAN?$AA?$AN?$AA?6?$AA?$AA@ 10003e98     esai_common_topaz_v1:mixerdrv.obj
 0001:00002eb0       ??_C@_1CE@NFMKBKIL@?$AAM?$AAX?$AAD?$AAM?$AA_?$AAG?$AAE?$AAT?$AAD?$AAE?$AAV?$AAC?$AAA?$AAP?$AAS?$AA?$AN?$AA?6?$AA?$AA@ 10003eb0     esai_common_topaz_v1:mixerdrv.obj
 0001:00002ed4       ??_C@_1CE@HLFFBCHG@?$AAM?$AAX?$AAD?$AAM?$AA_?$AAG?$AAE?$AAT?$AAN?$AAU?$AAM?$AAD?$AAE?$AAV?$AAS?$AA?$AN?$AA?6?$AA?$AA@ 10003ed4     esai_common_topaz_v1:mixerdrv.obj
 0001:00002ef8       ??_C@_1O@IKMMPJPA@?$AA?9?$AA?9?$AA?$CF?$AAs?$AA?$AN?$AA?6?$AA?$AA@ 10003ef8     spisdk_common_topaz_v1:spisdk.obj
 0001:00002f08       ??_C@_1DO@DICKCBEO@?$AA?$CF?$AAs?$AA?3?$AA?5?$AA?5?$AAC?$AAr?$AAe?$AAa?$AAt?$AAe?$AAF?$AAi?$AAl?$AAe?$AA?5?$AAC?$AAS?$AAP?$AAI?$AA?5?$AAf?$AAa?$AAi?$AAl?$AAe?$AAd?$AA?$CB?$AA?$AN?$AA?6?$AA?$AA@ 10003f08     spisdk_common_topaz_v1:spisdk.obj
 0001:00002f48       ??_C@_1O@JNDDBHKG@?$AA?$CL?$AA?$CL?$AA?$CF?$AAs?$AA?$AN?$AA?6?$AA?$AA@ 10003f48     spisdk_common_topaz_v1:spisdk.obj
 0001:00002f58       ??_C@_1BO@CGKLDFMN@?$AAC?$AAS?$AAP?$AAI?$AAO?$AAp?$AAe?$AAn?$AAH?$AAa?$AAn?$AAd?$AAl?$AAe?$AA?$AA@ 10003f58     spisdk_common_topaz_v1:spisdk.obj
 0001:00002f78       ??_C@_1DE@BBBAGJCD@?$AA?$CF?$AAs?$AA?3?$AA?5?$AAC?$AAl?$AAo?$AAs?$AAe?$AAH?$AAa?$AAn?$AAd?$AAl?$AAe?$AA?5?$AAf?$AAa?$AAi?$AAl?$AAe?$AAd?$AA?$CB?$AA?$AN?$AA?6?$AA?$AA@ 10003f78     spisdk_common_topaz_v1:spisdk.obj
 0001:00002fac       ??_C@_1CA@LFAHNJKO@?$AAC?$AAS?$AAP?$AAI?$AAC?$AAl?$AAo?$AAs?$AAe?$AAH?$AAa?$AAn?$AAd?$AAl?$AAe?$AA?$AA@ 10003fac     spisdk_common_topaz_v1:spisdk.obj
 0001:00002fd0       ??_C@_1EE@CKAHIHAM@?$AA?$CF?$AAs?$AA?3?$AA?5?$AAC?$AAS?$AAP?$AAI?$AA_?$AAI?$AAO?$AAC?$AAT?$AAL?$AA_?$AAE?$AAX?$AAC?$AAH?$AAA?$AAN?$AAG?$AAE?$AA?5?$AAf?$AAa?$AAi?$AAl?$AAe?$AAd?$AA?$CB?$AA?$AN@ 10003fd0     spisdk_common_topaz_v1:spisdk.obj
 0001:00003014       ??_C@_1BK@HGHKLBD@?$AAC?$AAS?$AAP?$AAI?$AAE?$AAx?$AAc?$AAh?$AAa?$AAn?$AAg?$AAe?$AA?$AA@ 10004014     spisdk_common_topaz_v1:spisdk.obj
 0001:00003030       ??_C@_1FC@LGELGOLM@?$AA?$CF?$AAs?$AA?3?$AA?5?$AAC?$AAS?$AAP?$AAI?$AA_?$AAI?$AAO?$AAC?$AAT?$AAL?$AA_?$AAE?$AAN?$AAA?$AAB?$AAL?$AAE?$AA_?$AAL?$AAO?$AAO?$AAP?$AAB?$AAA?$AAC?$AAK?$AA?5?$AAf@ 10004030     spisdk_common_topaz_v1:spisdk.obj
 0001:00003084       ??_C@_1CG@DPJCOMPP@?$AAC?$AAS?$AAP?$AAI?$AAE?$AAn?$AAa?$AAb?$AAl?$AAe?$AAL?$AAo?$AAo?$AAp?$AAb?$AAa?$AAc?$AAk?$AA?$AA@ 10004084     spisdk_common_topaz_v1:spisdk.obj
 0001:000030b0       ??_C@_1FE@FIIFDEJC@?$AA?$CF?$AAs?$AA?3?$AA?5?$AAC?$AAS?$AAP?$AAI?$AA_?$AAI?$AAO?$AAC?$AAT?$AAL?$AA_?$AAD?$AAI?$AAS?$AAA?$AAB?$AAL?$AAE?$AA_?$AAL?$AAO?$AAO?$AAP?$AAB?$AAA?$AAC?$AAK?$AA?5@ 100040b0     spisdk_common_topaz_v1:spisdk.obj
 0001:00003104       ??_C@_1CI@HELLEHFI@?$AAC?$AAS?$AAP?$AAI?$AAD?$AAi?$AAs?$AAa?$AAb?$AAl?$AAe?$AAL?$AAo?$AAo?$AAp?$AAb?$AAa?$AAc?$AAk?$AA?$AA@ 10004104     spisdk_common_topaz_v1:spisdk.obj
 0001:00003130       ??_C@_1FO@JNLAMKFK@?$AA?$CK?$AA?$CK?$AA?$CK?$AA?$CK?$AA?$CK?$AA?5?$AAD?$AAL?$AAL?$AA?5?$AAP?$AAR?$AAO?$AAC?$AAE?$AAS?$AAS?$AA?5?$AAD?$AAE?$AAT?$AAA?$AAC?$AAH?$AA?5?$AAF?$AAR?$AAO?$AAM?$AA?5?$AAC?$AAS@ 10004130     spisdk_common_topaz_v1:spisdk.obj
 0001:00003190       ??_C@_1FK@JFLMINEA@?$AA?$CK?$AA?$CK?$AA?$CK?$AA?$CK?$AA?$CK?$AA?5?$AAD?$AAL?$AAL?$AA?5?$AAP?$AAR?$AAO?$AAC?$AAE?$AAS?$AAS?$AA?5?$AAA?$AAT?$AAT?$AAA?$AAC?$AAH?$AA?5?$AAT?$AAO?$AA?5?$AAC?$AAS?$AAP?$AAI@ 10004190     spisdk_common_topaz_v1:spisdk.obj
 0001:00003214       ??0CWM8580@@QAA@XZ         10004214 f   wm8580.obj
 0001:0000329c       ??1CWM8580@@QAA@XZ         1000429c f   wm8580.obj
 0001:000032bc       ?ReadRegister@CWM8580@@AAAEK@Z 100042bc f   wm8580.obj
 0001:000033e8       ?WriteRegister@CWM8580@@AAAHKK@Z 100043e8 f   wm8580.obj
 0001:00003520       ?InitCodec@CWM8580@@QAAHXZ 10004520 f   wm8580.obj
 0001:000035c0       ?GetDeviceID@CWM8580@@QAAHXZ 100045c0 f   wm8580.obj
 0001:00003638       ?ConfigOutput@CWM8580@@QAAHKKKKW4AUDIO_PROTOCOL@@@Z 10004638 f   wm8580.obj
 0001:00003c5c       ?EnableDAC@CWM8580@@QAAHXZ 10004c5c f   wm8580.obj
 0001:00003d10       ?DisableDAC@CWM8580@@QAAHXZ 10004d10 f   wm8580.obj
 0001:00003d98       ?SetOutputGain@CWM8580@@QAAHKKKK@Z 10004d98 f   wm8580.obj
 0001:00003ebc       ?SetOutputMute@CWM8580@@QAAHHK@Z 10004ebc f   wm8580.obj
 0001:00003ee4       ?GetDACBitClock@CWM8580@@QAAIXZ 10004ee4 f   wm8580.obj
 0001:00004028       ?EnableCLKO@CWM8580@@QAAHXZ 10005028 f   wm8580.obj
 0001:00004214       ??0CAK5702@@QAA@XZ         10005214 f   ak5702.obj
 0001:00004324       ??1CAK5702@@QAA@XZ         10005324 f   ak5702.obj
 0001:00004344       ?ReadRegister@CAK5702@@AAAEE@Z 10005344 f   ak5702.obj
 0001:00004464       ?WriteRegister@CAK5702@@AAAHEE@Z 10005464 f   ak5702.obj
 0001:0000454c       ?DumpRegs@CAK5702@@AAAXXZ  1000554c f   ak5702.obj
 0001:00004560       ?InitAK5702@CAK5702@@QAAHXZ 10005560 f   ak5702.obj
 0001:00004700       ?ConfigADC@CAK5702@@QAAHW4AUDIO_PROTOCOL@@KKKKW4AK5702_PLL_MODE@@@Z 10005700 f   ak5702.obj
 0001:00004a78       ?EnalbeADC@CAK5702@@QAAHXZ 10005a78 f   ak5702.obj
 0001:00004c3c       ?DisableADC@CAK5702@@QAAHXZ 10005c3c f   ak5702.obj
 0001:00004d40       ?SetPLLPower@CAK5702@@QAAXH@Z 10005d40 f   ak5702.obj
 0001:00004e24       ?SetCodecPower@CAK5702@@QAAXW4AK5702_POWER_MODE@@@Z 10005e24 f   ak5702.obj
 0001:00004fac       ?SetInputGain@CAK5702@@QAAXEEEEK@Z 10005fac f   ak5702.obj
 0001:00005048       ?BSPAudioInitCodec@@YAHXZ  10006048 f   bsphwctxt.obj
 0001:00005204       ?BSPAudioConfigDAC@@YAHKKKKW4AUDIO_PROTOCOL@@@Z 10006204 f   bsphwctxt.obj
 0001:00005258       ?BSPAudioConfigADC@@YAHKKKKW4AUDIO_PROTOCOL@@@Z 10006258 f   bsphwctxt.obj
 0001:000052b4       ?BSPAudioDeinitCodec@@YAXXZ 100062b4 f   bsphwctxt.obj
 0001:00005388       ?BSPAudioStartDAC@@YAXXZ   10006388 f   bsphwctxt.obj
 0001:000053a4       ?BSPAudioStopDAC@@YAXXZ    100063a4 f   bsphwctxt.obj
 0001:000053c0       ?BSPAudioStartADC@@YAXXZ   100063c0 f   bsphwctxt.obj
 0001:000053dc       ?BSPAudioStopADC@@YAXXZ    100063dc f   bsphwctxt.obj
 0001:000053f8       ?BSPAudioSetOutputGain@@YAXK@Z 100063f8 f   bsphwctxt.obj
 0001:00005438       ?BSPAudioSetInputGain@@YAXK@Z 10006438 f   bsphwctxt.obj
 0001:000054c0       ?BSPAudioGetInputDeviceNum@@YAEXZ 100064c0 f   bsphwctxt.obj
 0001:000054d8       ?BSPAllocOutputDMABuffer@@YAGPAPAEPAT_LARGE_INTEGER@@@Z 100064d8 f   bsphwctxt.obj
 0001:00005544       ?BSPDeallocOutputDMABuffer@@YAXPAET_LARGE_INTEGER@@@Z 10006544 f   bsphwctxt.obj
 0001:000055a4       ?BSPAllocInputDMABuffer@@YAGPAPAEPAT_LARGE_INTEGER@@@Z 100065a4 f   bsphwctxt.obj
 0001:00005610       ?BSPDeallocInputDMABuffer@@YAXPAET_LARGE_INTEGER@@@Z 10006610 f   bsphwctxt.obj
 0001:00005670       ?BSPAudioIomuxConfig@@YAXXZ 10006670 f   bsphwctxt.obj
 0001:0000573c       ?BSPESAIEnableClock@@YAHIH@Z 1000673c f   bsphwctxt.obj
 0001:000057d0       ?BSPAudioGetSdmaPriority@@YAEXZ 100067d0 f   bsphwctxt.obj
 0001:000057e8       ?BSPAudioPowerUp@@YAXH@Z   100067e8 f   bsphwctxt.obj
 0001:000057fc       ?BSPAudioPowerDown@@YAXH@Z 100067fc f   bsphwctxt.obj
 0001:00005810       ?BSPAudioGetOutputProtocol@@YA?AW4AUDIO_PROTOCOL@@XZ 10006810 f   bsphwctxt.obj
 0001:00005830       ?BSPAudioGetInputProtocol@@YA?AW4AUDIO_PROTOCOL@@XZ 10006830 f   bsphwctxt.obj
 0001:00005850       ?BSPIsSupportedOutputFormat@@YAHPAUWAVEFORMATEXTENSIBLE@@@Z 10006850 f   bsphwctxt.obj
 0001:00005f44       ?BSPIsSupportedInputFormat@@YAHPAUWAVEFORMATEXTENSIBLE@@@Z 10006f44 f   bsphwctxt.obj
 0001:000063c8       ?BSPAudioGetTxBitClock@@YAIXZ 100073c8 f   bsphwctxt.obj
 0001:000063fc       ??_GCWM8580@@QAAPAXI@Z     100073fc f i bsphwctxt.obj
 0001:00006440       ??_GCAK5702@@QAAPAXI@Z     10007440 f i bsphwctxt.obj
 0001:00006484       DllMain                    10007484 f   esai_common_topaz_v1:wavemain.obj
 0001:000064d4       WAV_Init                   100074d4 f   esai_common_topaz_v1:wavemain.obj
 0001:00006508       WAV_Deinit                 10007508 f   esai_common_topaz_v1:wavemain.obj
 0001:00006544       WAV_Open                   10007544 f   esai_common_topaz_v1:wavemain.obj
 0001:000065ac       WAV_Close                  100075ac f   esai_common_topaz_v1:wavemain.obj
 0001:000065ec       ?HandleWaveMessage@@YAHPAUMMDRV_MESSAGE_PARAMS@@PAK@Z 100075ec f   esai_common_topaz_v1:wavemain.obj
 0001:00006e8c       WAV_IOControl              10007e8c f   esai_common_topaz_v1:wavemain.obj
 0001:00007044       ?Lock@HardwareContext@@QAAXXZ 10008044 f i esai_common_topaz_v1:wavemain.obj
 0001:00007064       ?Unlock@HardwareContext@@QAAXXZ 10008064 f i esai_common_topaz_v1:wavemain.obj
 0001:00007084       ?GetNumInputDevices@HardwareContext@@QAAKXZ 10008084 f i esai_common_topaz_v1:wavemain.obj
 0001:000070b4       ?GetNumOutputDevices@HardwareContext@@QAAKXZ 100080b4 f i esai_common_topaz_v1:wavemain.obj
 0001:000070dc       ?GetInputDeviceContext@HardwareContext@@QAAPAVDeviceContext@@I@Z 100080dc f i esai_common_topaz_v1:wavemain.obj
 0001:00007108       ?GetOutputDeviceContext@HardwareContext@@QAAPAVDeviceContext@@I@Z 10008108 f i esai_common_topaz_v1:wavemain.obj
 0001:00007134       ?CreateHWContext@HardwareContext@@SAHK@Z 10008134 f   esai_common_topaz_v1:hwctxt.obj
 0001:000071f8       ??0HardwareContext@@QAA@XZ 100081f8 f   esai_common_topaz_v1:hwctxt.obj
 0001:0000726c       ??1HardwareContext@@QAA@XZ 1000826c f   esai_common_topaz_v1:hwctxt.obj
 0001:0000728c       ?Init@HardwareContext@@QAAHK@Z 1000828c f   esai_common_topaz_v1:hwctxt.obj
 0001:0000768c       ?Deinit@HardwareContext@@QAAHXZ 1000868c f   esai_common_topaz_v1:hwctxt.obj
 0001:000077a0       ?DumpESAIRegs@HardwareContext@@AAAXXZ 100087a0 f   esai_common_topaz_v1:hwctxt.obj
 0001:000077b4       ?InitESAI@HardwareContext@@AAAXXZ 100087b4 f   esai_common_topaz_v1:hwctxt.obj
 0001:00007824       ?ConfigESAITx@HardwareContext@@AAAXXZ 10008824 f   esai_common_topaz_v1:hwctxt.obj
 0001:00007a80       ?ConfigESAIRx@HardwareContext@@AAAXXZ 10008a80 f   esai_common_topaz_v1:hwctxt.obj
 0001:00007ca4       ?InitOutputDMA@HardwareContext@@AAAHXZ 10008ca4 f   esai_common_topaz_v1:hwctxt.obj
 0001:00007ef0       ?ConfigOutputDMA@HardwareContext@@AAAHXZ 10008ef0 f   esai_common_topaz_v1:hwctxt.obj
 0001:00008104       ?InitInputDMA@HardwareContext@@AAAHXZ 10009104 f   esai_common_topaz_v1:hwctxt.obj
 0001:00008394       ?ConfigInputDMA@HardwareContext@@AAAHXZ 10009394 f   esai_common_topaz_v1:hwctxt.obj
 0001:000085cc       ?InitInterruptThread@HardwareContext@@IAAHXZ 100095cc f   esai_common_topaz_v1:hwctxt.obj
 0001:000086f8       ?InitDisableDelayThread@HardwareContext@@IAAHXZ 100096f8 f   esai_common_topaz_v1:hwctxt.obj
 0001:00008940       ?StartCodec@HardwareContext@@AAAXW4AUDIO_BUS@@@Z 10009940 f   esai_common_topaz_v1:hwctxt.obj
 0001:0000896c       ?StopCodec@HardwareContext@@AAAXW4AUDIO_BUS@@@Z 1000996c f   esai_common_topaz_v1:hwctxt.obj
 0001:00008aa0       ?PrepareESAI@HardwareContext@@AAAXW4AUDIO_BUS@@@Z 10009aa0 f   esai_common_topaz_v1:hwctxt.obj
 0001:00008d0c       ?StartESAI@HardwareContext@@AAAXW4AUDIO_BUS@@@Z 10009d0c f   esai_common_topaz_v1:hwctxt.obj
 0001:00008f74       ?StopESAI@HardwareContext@@AAAXW4AUDIO_BUS@@@Z 10009f74 f   esai_common_topaz_v1:hwctxt.obj
 0001:000091b8       ?StartOutputDMA@HardwareContext@@QAAHXZ 1000a1b8 f   esai_common_topaz_v1:hwctxt.obj
 0001:0000947c       ?StopOutputDMA@HardwareContext@@QAAXXZ 1000a47c f   esai_common_topaz_v1:hwctxt.obj
 0001:00009544       ?StartInputDMA@HardwareContext@@QAAHXZ 1000a544 f   esai_common_topaz_v1:hwctxt.obj
 0001:000096d4       ?StopInputDMA@HardwareContext@@QAAXXZ 1000a6d4 f   esai_common_topaz_v1:hwctxt.obj
 0001:0000975c       ?TransferOutputBuffers@HardwareContext@@IAAKXZ 1000a75c f   esai_common_topaz_v1:hwctxt.obj
 0001:00009854       ?TransferInputBuffers@HardwareContext@@IAAKE@Z 1000a854 f   esai_common_topaz_v1:hwctxt.obj
 0001:000099e4       ?TransferBuffer@HardwareContext@@IAAKW4AUDIO_BUS@@E@Z 1000a9e4 f   esai_common_topaz_v1:hwctxt.obj
 0001:00009b44       ?InterruptThread@HardwareContext@@QAAXXZ 1000ab44 f   esai_common_topaz_v1:hwctxt.obj
 0001:00009c18       ?OutputIntrRoutine@HardwareContext@@AAAXXZ 1000ac18 f   esai_common_topaz_v1:hwctxt.obj
 0001:00009eb0       ?InputIntrRoutine@HardwareContext@@AAAXXZ 1000aeb0 f   esai_common_topaz_v1:hwctxt.obj
 0001:0000a200       ?DisableDelayThread@HardwareContext@@QAAXXZ 1000b200 f   esai_common_topaz_v1:hwctxt.obj
 0001:0000a454       ?CallInterruptThread@@YAXPAVHardwareContext@@@Z 1000b454 f   esai_common_topaz_v1:hwctxt.obj
 0001:0000a470       ?CallDisableDelayThread@@YAXPAVHardwareContext@@@Z 1000b470 f   esai_common_topaz_v1:hwctxt.obj
 0001:0000a48c       ?SetOutputGain@HardwareContext@@QAAIK@Z 1000b48c f   esai_common_topaz_v1:hwctxt.obj
 0001:0000a4cc       ?SetOutputMute@HardwareContext@@QAAIH@Z 1000b4cc f   esai_common_topaz_v1:hwctxt.obj
 0001:0000a50c       ?GetOutputGain@HardwareContext@@QAAKXZ 1000b50c f   esai_common_topaz_v1:hwctxt.obj
 0001:0000a53c       ?GetOutputMute@HardwareContext@@QAAHXZ 1000b53c f   esai_common_topaz_v1:hwctxt.obj
 0001:0000a56c       ?GetInputMute@HardwareContext@@QAAHXZ 1000b56c f   esai_common_topaz_v1:hwctxt.obj
 0001:0000a59c       ?SetInputMute@HardwareContext@@QAAIH@Z 1000b59c f   esai_common_topaz_v1:hwctxt.obj
 0001:0000a5dc       ?GetInputGain@HardwareContext@@QAAKXZ 1000b5dc f   esai_common_topaz_v1:hwctxt.obj
 0001:0000a60c       ?SetInputGain@HardwareContext@@QAAIK@Z 1000b60c f   esai_common_topaz_v1:hwctxt.obj
 0001:0000a64c       ?PmControlMessage@HardwareContext@@QAAHKPAEK0KPAK@Z 1000b64c f   esai_common_topaz_v1:hwctxt.obj
 0001:0000a818       ?PowerUp@HardwareContext@@QAAXXZ 1000b818 f   esai_common_topaz_v1:hwctxt.obj
 0001:0000a87c       ?PowerDown@HardwareContext@@QAAXXZ 1000b87c f   esai_common_topaz_v1:hwctxt.obj
 0001:0000a930       ?GetDriverRegValue@HardwareContext@@QAAKPAGK@Z 1000b930 f   esai_common_topaz_v1:hwctxt.obj
 0001:0000a9b4       ?SetDriverRegValue@HardwareContext@@QAAXPAGK@Z 1000b9b4 f   esai_common_topaz_v1:hwctxt.obj
 0001:0000aa24       ?IsSupportedOutputFormat@HardwareContext@@QAAHPAUtWAVEFORMATEX@@@Z 1000ba24 f   esai_common_topaz_v1:hwctxt.obj
 0001:0000ab4c       ?IsSupportedInputFormat@HardwareContext@@QAAHPAUtWAVEFORMATEX@@@Z 1000bb4c f   esai_common_topaz_v1:hwctxt.obj
 0001:0000ac04       ?InitOutputWaveFormat@HardwareContext@@QAAHPAUtWAVEFORMATEX@@@Z 1000bc04 f   esai_common_topaz_v1:hwctxt.obj
 0001:0000aeac       ?InitInputWaveFormat@HardwareContext@@QAAHPAUtWAVEFORMATEX@@@Z 1000beac f   esai_common_topaz_v1:hwctxt.obj
 0001:0000aff4       ?DeinitInputWaveFormat@HardwareContext@@QAAHPAUtWAVEFORMATEX@@@Z 1000bff4 f   esai_common_topaz_v1:hwctxt.obj
 0001:0000b02c       ?DeinitOutputWaveFormat@HardwareContext@@QAAHPAUtWAVEFORMATEX@@@Z 1000c02c f   esai_common_topaz_v1:hwctxt.obj
 0001:0000b064       ?ForceSpeaker@HardwareContext@@QAAKH@Z 1000c064 f   esai_common_topaz_v1:hwctxt.obj
 0001:0000b08c       ?SelectInputSource@HardwareContext@@QAAHK@Z 1000c08c f   esai_common_topaz_v1:hwctxt.obj
 0001:0000b0b4       ?CallAsrcIntrThread@@YAXPAVHardwareContext@@@Z 1000c0b4 f   esai_common_topaz_v1:hwctxt.obj
 0001:0000b0d0       ?AsrcIntrThread@HardwareContext@@QAAXXZ 1000c0d0 f   esai_common_topaz_v1:hwctxt.obj
 0001:0000b204       ?AsrcIntrRoutine@HardwareContext@@AAAXXZ 1000c204 f   esai_common_topaz_v1:hwctxt.obj
 0001:0000b418       ?InitAsrcP2P@HardwareContext@@AAAHXZ 1000c418 f   esai_common_topaz_v1:hwctxt.obj
 0001:0000b734       ?DeinitAsrcP2P@HardwareContext@@AAAXXZ 1000c734 f   esai_common_topaz_v1:hwctxt.obj
 0001:0000b7c4       ?ConfigAsrc@HardwareContext@@AAAHXZ 1000c7c4 f   esai_common_topaz_v1:hwctxt.obj
 0001:0000ba94       ??0InputDeviceContext@@QAA@XZ 1000ca94 f i esai_common_topaz_v1:hwctxt.obj
 0001:0000bad4       ??0OutputDeviceContext@@QAA@XZ 1000cad4 f i esai_common_topaz_v1:hwctxt.obj
 0001:0000bb14       SetEvent                   1000cb14 f i esai_common_topaz_v1:hwctxt.obj
 0001:0000bb4c       ?GetInterruptThreadPriority@HardwareContext@@IAAKXZ 1000cb4c f i esai_common_topaz_v1:hwctxt.obj
 0001:0000bb8c       ?UpdateOutputGain@HardwareContext@@IAAXXZ 1000cb8c f i esai_common_topaz_v1:hwctxt.obj
 0001:0000bbe0       ?UpdateInputGain@HardwareContext@@IAAXXZ 1000cbe0 f i esai_common_topaz_v1:hwctxt.obj
 0001:0000bc34       PulseEvent                 1000cc34 f i esai_common_topaz_v1:hwctxt.obj
 0001:0000bc6c       ??0DeviceContext@@QAA@XZ   1000cc6c f   esai_common_topaz_v1:devctxt.obj
 0001:0000bd48       ?GetGain@DeviceContext@@QAAKXZ 1000cd48 f   esai_common_topaz_v1:devctxt.obj
 0001:0000bd78       ?SetGain@DeviceContext@@QAAKK@Z 1000cd78 f   esai_common_topaz_v1:devctxt.obj
 0001:0000bdb8       ?GetDefaultStreamGain@DeviceContext@@QAAKXZ 1000cdb8 f   esai_common_topaz_v1:devctxt.obj
 0001:0000bde8       ?SetDefaultStreamGain@DeviceContext@@QAAKK@Z 1000cde8 f   esai_common_topaz_v1:devctxt.obj
 0001:0000be20       ?GetSecondaryGainLimit@DeviceContext@@QAAKK@Z 1000ce20 f   esai_common_topaz_v1:devctxt.obj
 0001:0000be60       ?SetSecondaryGainLimit@DeviceContext@@QAAKKK@Z 1000ce60 f   esai_common_topaz_v1:devctxt.obj
 0001:0000bec8       ?IsSupportedFormat@DeviceContext@@UAAHPAUtWAVEFORMATEX@@@Z 1000cec8 f   esai_common_topaz_v1:devctxt.obj
 0001:0000c068       ?IsSupportedFormat@OutputDeviceContext@@UAAHPAUtWAVEFORMATEX@@@Z 1000d068 f   esai_common_topaz_v1:devctxt.obj
 0001:0000c100       ?IsSupportedFormat@InputDeviceContext@@UAAHPAUtWAVEFORMATEX@@@Z 1000d100 f   esai_common_topaz_v1:devctxt.obj
 0001:0000c158       ?DeinitDeviceWaveFormat@DeviceContext@@UAAHPAUtWAVEFORMATEX@@@Z 1000d158 f   esai_common_topaz_v1:devctxt.obj
 0001:0000c180       ?DeinitDeviceWaveFormat@OutputDeviceContext@@UAAHPAUtWAVEFORMATEX@@@Z 1000d180 f   esai_common_topaz_v1:devctxt.obj
 0001:0000c1c0       ?DeinitDeviceWaveFormat@InputDeviceContext@@UAAHPAUtWAVEFORMATEX@@@Z 1000d1c0 f   esai_common_topaz_v1:devctxt.obj
 0001:0000c200       ?InitDeviceWaveFormat@DeviceContext@@UAAHPAUtWAVEFORMATEX@@@Z 1000d200 f   esai_common_topaz_v1:devctxt.obj
 0001:0000c228       ?InitDeviceWaveFormat@OutputDeviceContext@@UAAHPAUtWAVEFORMATEX@@@Z 1000d228 f   esai_common_topaz_v1:devctxt.obj
 0001:0000c268       ?InitDeviceWaveFormat@InputDeviceContext@@UAAHPAUtWAVEFORMATEX@@@Z 1000d268 f   esai_common_topaz_v1:devctxt.obj
 0001:0000c2a8       ?NewStream@DeviceContext@@UAAKPAVStreamContext@@@Z 1000d2a8 f   esai_common_topaz_v1:devctxt.obj
 0001:0000c3ec       ?DeleteStream@DeviceContext@@QAAXPAVStreamContext@@@Z 1000d3ec f   esai_common_topaz_v1:devctxt.obj
 0001:0000c4a4       ?TransferBuffer@DeviceContext@@QAAPAEPAE0PAUTRANSFER_STATUS@@@Z 1000d4a4 f   esai_common_topaz_v1:devctxt.obj
 0001:0000c5b4       ?RecalcAllGains@DeviceContext@@QAAXXZ 1000d5b4 f   esai_common_topaz_v1:devctxt.obj
 0001:0000c630       ?StreamReadyToRender@OutputDeviceContext@@UAAXPAVStreamContext@@@Z 1000d630 f   esai_common_topaz_v1:devctxt.obj
 0001:0000c654       ?StreamReadyToRender@InputDeviceContext@@UAAXPAVStreamContext@@@Z 1000d654 f   esai_common_topaz_v1:devctxt.obj
 0001:0000c678       ?GetDevCaps@OutputDeviceContext@@UAAKPAXK@Z 1000d678 f   esai_common_topaz_v1:devctxt.obj
 0001:0000c6c8       ?GetDevCaps@InputDeviceContext@@UAAKPAXK@Z 1000d6c8 f   esai_common_topaz_v1:devctxt.obj
 0001:0000c718       ?GetExtDevCaps@OutputDeviceContext@@UAAKPAXK@Z 1000d718 f   esai_common_topaz_v1:devctxt.obj
 0001:0000c768       ?GetExtDevCaps@InputDeviceContext@@UAAKPAXK@Z 1000d768 f   esai_common_topaz_v1:devctxt.obj
 0001:0000c790       ?CreateStream@InputDeviceContext@@UAAPAVStreamContext@@PAUwaveopendesc_tag@@@Z 1000d790 f   esai_common_topaz_v1:devctxt.obj
 0001:0000c854       ?CreateStream@OutputDeviceContext@@UAAPAVStreamContext@@PAUwaveopendesc_tag@@@Z 1000d854 f   esai_common_topaz_v1:devctxt.obj
 0001:0000cb78       ?OpenStream@DeviceContext@@QAAKPAUwaveopendesc_tag@@KPAPAVStreamContext@@@Z 1000db78 f   esai_common_topaz_v1:devctxt.obj
 0001:0000cdcc       ?SetBaseSampleRate@DeviceContext@@UAAXK@Z 1000ddcc f   esai_common_topaz_v1:devctxt.obj
 0001:0000ce1c       ?ResetBaseInfo@DeviceContext@@QAAXXZ 1000de1c f   esai_common_topaz_v1:devctxt.obj
 0001:0000ce98       ?GetBaseSampleRate@DeviceContext@@QAAKXZ 1000de98 f   esai_common_topaz_v1:devctxt.obj
 0001:0000cec8       ?GetBaseSampleRateInverse@DeviceContext@@QAAKXZ 1000dec8 f   esai_common_topaz_v1:devctxt.obj
 0001:0000cef8       ?GetChannels@OutputDeviceContext@@UAAKXZ 1000def8 f   esai_common_topaz_v1:devctxt.obj
 0001:0000cf20       ?GetChannels@InputDeviceContext@@UAAKXZ 1000df20 f   esai_common_topaz_v1:devctxt.obj
 0001:0000cf48       ?GetNativeFormat@DeviceContext@@QAAKKPAXKPAK@Z 1000df48 f   esai_common_topaz_v1:devctxt.obj
 0001:0000d078       ?GetProperty@DeviceContext@@QAAKPAUtag_WAVEPROPINFO@@@Z 1000e078 f   esai_common_topaz_v1:devctxt.obj
 0001:0000d1c8       ?SetProperty@DeviceContext@@QAAKPAUtag_WAVEPROPINFO@@@Z 1000e1c8 f   esai_common_topaz_v1:devctxt.obj
 0001:0000d1f8       ??0InputStreamContextEx@@QAA@XZ 1000e1f8 f i esai_common_topaz_v1:devctxt.obj
 0001:0000d23c       ??_GInputStreamContextEx@@UAAPAXI@Z 1000e23c f i esai_common_topaz_v1:devctxt.obj
 0001:0000d23c       ??_EInputStreamContextEx@@UAAPAXI@Z 1000e23c f i esai_common_topaz_v1:devctxt.obj
 0001:0000d280       ??0InputStreamContext@@QAA@XZ 1000e280 f i esai_common_topaz_v1:devctxt.obj
 0001:0000d2c4       ??1InputStreamContextEx@@UAA@XZ 1000e2c4 f i esai_common_topaz_v1:devctxt.obj
 0001:0000d2e0       ??1InputStreamContext@@UAA@XZ 1000e2e0 f i esai_common_topaz_v1:devctxt.obj
 0001:0000d2fc       ??_GInputStreamContext@@UAAPAXI@Z 1000e2fc f i esai_common_topaz_v1:devctxt.obj
 0001:0000d2fc       ??_EInputStreamContext@@UAAPAXI@Z 1000e2fc f i esai_common_topaz_v1:devctxt.obj
 0001:0000d340       ??0WaveStreamContext@@QAA@XZ 1000e340 f i esai_common_topaz_v1:devctxt.obj
 0001:0000d384       ??1WaveStreamContext@@UAA@XZ 1000e384 f i esai_common_topaz_v1:devctxt.obj
 0001:0000d3a0       ??_EWaveStreamContext@@UAAPAXI@Z 1000e3a0 f i esai_common_topaz_v1:devctxt.obj
 0001:0000d3a0       ??_GWaveStreamContext@@UAAPAXI@Z 1000e3a0 f i esai_common_topaz_v1:devctxt.obj
 0001:0000d3e4       ??0OutputStreamContextEx@@QAA@XZ 1000e3e4 f i esai_common_topaz_v1:devctxt.obj
 0001:0000d428       ??0OutputStreamContextM8@@QAA@XZ 1000e428 f i esai_common_topaz_v1:devctxt.obj
 0001:0000d46c       ??0OutputStreamContextS8@@QAA@XZ 1000e46c f i esai_common_topaz_v1:devctxt.obj
 0001:0000d4b0       ??0OutputStreamContextM16@@QAA@XZ 1000e4b0 f i esai_common_topaz_v1:devctxt.obj
 0001:0000d4f4       ??0OutputStreamContextS16@@QAA@XZ 1000e4f4 f i esai_common_topaz_v1:devctxt.obj
 0001:0000d538       ??_GOutputStreamContextEx@@UAAPAXI@Z 1000e538 f i esai_common_topaz_v1:devctxt.obj
 0001:0000d538       ??_EOutputStreamContextEx@@UAAPAXI@Z 1000e538 f i esai_common_topaz_v1:devctxt.obj
 0001:0000d57c       ??0OutputStreamContext@@QAA@XZ 1000e57c f i esai_common_topaz_v1:devctxt.obj
 0001:0000d5c0       ??_EOutputStreamContextM8@@UAAPAXI@Z 1000e5c0 f i esai_common_topaz_v1:devctxt.obj
 0001:0000d5c0       ??_GOutputStreamContextM8@@UAAPAXI@Z 1000e5c0 f i esai_common_topaz_v1:devctxt.obj
 0001:0000d604       ??_EOutputStreamContextS8@@UAAPAXI@Z 1000e604 f i esai_common_topaz_v1:devctxt.obj
 0001:0000d604       ??_GOutputStreamContextS8@@UAAPAXI@Z 1000e604 f i esai_common_topaz_v1:devctxt.obj
 0001:0000d648       ??_EOutputStreamContextM16@@UAAPAXI@Z 1000e648 f i esai_common_topaz_v1:devctxt.obj
 0001:0000d648       ??_GOutputStreamContextM16@@UAAPAXI@Z 1000e648 f i esai_common_topaz_v1:devctxt.obj
 0001:0000d68c       ??_GOutputStreamContextS16@@UAAPAXI@Z 1000e68c f i esai_common_topaz_v1:devctxt.obj
 0001:0000d68c       ??_EOutputStreamContextS16@@UAAPAXI@Z 1000e68c f i esai_common_topaz_v1:devctxt.obj
 0001:0000d6d0       ??1OutputStreamContextEx@@UAA@XZ 1000e6d0 f i esai_common_topaz_v1:devctxt.obj
 0001:0000d6ec       ??1OutputStreamContext@@UAA@XZ 1000e6ec f i esai_common_topaz_v1:devctxt.obj
 0001:0000d708       ??_EOutputStreamContext@@UAAPAXI@Z 1000e708 f i esai_common_topaz_v1:devctxt.obj
 0001:0000d708       ??_GOutputStreamContext@@UAAPAXI@Z 1000e708 f i esai_common_topaz_v1:devctxt.obj
 0001:0000d74c       ??1OutputStreamContextM8@@UAA@XZ 1000e74c f i esai_common_topaz_v1:devctxt.obj
 0001:0000d768       ??1OutputStreamContextS8@@UAA@XZ 1000e768 f i esai_common_topaz_v1:devctxt.obj
 0001:0000d784       ??1OutputStreamContextM16@@UAA@XZ 1000e784 f i esai_common_topaz_v1:devctxt.obj
 0001:0000d7a0       ??1OutputStreamContextS16@@UAA@XZ 1000e7a0 f i esai_common_topaz_v1:devctxt.obj
 0001:0000d7bc       ?IsEqualGUID@@YAHABU_GUID@@0@Z 1000e7bc f i esai_common_topaz_v1:devctxt.obj
 0001:0000d818       ??0StreamContext@@QAA@XZ   1000e818 f   esai_common_topaz_v1:strmctxt.obj
 0001:0000d850       ??1StreamContext@@UAA@XZ   1000e850 f   esai_common_topaz_v1:strmctxt.obj
 0001:0000d874       ?StillPlaying@StreamContext@@QAAHXZ 1000e874 f   esai_common_topaz_v1:strmctxt.obj
 0001:0000d8c4       ?GetByteCount@StreamContext@@QAAKXZ 1000e8c4 f   esai_common_topaz_v1:strmctxt.obj
 0001:0000d8f4       ?GetWaveFormat@StreamContext@@QAAPAUtWAVEFORMATEX@@XZ 1000e8f4 f   esai_common_topaz_v1:strmctxt.obj
 0001:0000d920       ?GetDeviceContext@StreamContext@@QAAPAVDeviceContext@@XZ 1000e920 f   esai_common_topaz_v1:strmctxt.obj
 0001:0000d950       ?DoDriverCallback@StreamContext@@QAAXIKK@Z 1000e950 f   esai_common_topaz_v1:strmctxt.obj
 0001:0000d9a8       ?DoCallbackReturnBuffer@StreamContext@@UAAXPAUwavehdr_tag@@@Z 1000e9a8 f   esai_common_topaz_v1:strmctxt.obj
 0001:0000d9d4       ?DoCallbackStreamOpened@StreamContext@@UAAXXZ 1000e9d4 f   esai_common_topaz_v1:strmctxt.obj
 0001:0000da00       ?DoCallbackStreamClosed@StreamContext@@UAAXXZ 1000ea00 f   esai_common_topaz_v1:strmctxt.obj
 0001:0000da28       ?ReturnBuffer@StreamContext@@QAAXPAUwavehdr_tag@@@Z 1000ea28 f   esai_common_topaz_v1:strmctxt.obj
 0001:0000da98       ?GetGain@StreamContext@@QAAKXZ 1000ea98 f   esai_common_topaz_v1:strmctxt.obj
 0001:0000dac8       ?SetGain@StreamContext@@QAAKK@Z 1000eac8 f   esai_common_topaz_v1:strmctxt.obj
 0001:0000db1c       ?SetSecondaryGainClass@StreamContext@@QAAKK@Z 1000eb1c f   esai_common_topaz_v1:strmctxt.obj
 0001:0000db88       ?GainChange@StreamContext@@UAAXXZ 1000eb88 f   esai_common_topaz_v1:strmctxt.obj
 0001:0000dc08       ?IsExclusive@StreamContext@@UAAHXZ 1000ec08 f   esai_common_topaz_v1:strmctxt.obj
 0001:0000dc30       ?Open@StreamContext@@UAAKPAVDeviceContext@@PAUwaveopendesc_tag@@K@Z 1000ec30 f   esai_common_topaz_v1:strmctxt.obj
 0001:0000dec0       ?Close@StreamContext@@UAAKXZ 1000eec0 f   esai_common_topaz_v1:strmctxt.obj
 0001:0000df34       ?AddRef@StreamContext@@QAAJXZ 1000ef34 f   esai_common_topaz_v1:strmctxt.obj
 0001:0000df88       ?Release@StreamContext@@QAAJXZ 1000ef88 f   esai_common_topaz_v1:strmctxt.obj
 0001:0000e04c       ?QueueBuffer@StreamContext@@UAAKPAUwavehdr_tag@@@Z 1000f04c f   esai_common_topaz_v1:strmctxt.obj
 0001:0000e20c       ?GetNextBuffer@StreamContext@@QAAPAEXZ 1000f20c f   esai_common_topaz_v1:strmctxt.obj
 0001:0000e3ec       ?BreakLoop@StreamContext@@QAAKXZ 1000f3ec f   esai_common_topaz_v1:strmctxt.obj
 0001:0000e4d0       ?MapGain@StreamContext@@QAAKKK@Z 1000f4d0 f   esai_common_topaz_v1:strmctxt.obj
 0001:0000e6e4       ?GetPos@StreamContext@@UAAKPAUmmtime_tag@@@Z 1000f6e4 f   esai_common_topaz_v1:strmctxt.obj
 0001:0000e918       ?Open@WaveStreamContext@@UAAKPAVDeviceContext@@PAUwaveopendesc_tag@@K@Z 1000f918 f   esai_common_topaz_v1:strmctxt.obj
 0001:0000eb3c       ?GetRate@WaveStreamContext@@QAAKPAK@Z 1000fb3c f   esai_common_topaz_v1:strmctxt.obj
 0001:0000eb78       ?Run@StreamContext@@UAAKXZ 1000fb78 f   esai_common_topaz_v1:strmctxt.obj
 0001:0000ebf4       ?Stop@StreamContext@@UAAKXZ 1000fbf4 f   esai_common_topaz_v1:strmctxt.obj
 0001:0000ec2c       ?Reset@StreamContext@@UAAKXZ 1000fc2c f   esai_common_topaz_v1:strmctxt.obj
 0001:0000ed40       ?ForceSpeaker@StreamContext@@QAAKH@Z 1000fd40 f   esai_common_topaz_v1:strmctxt.obj
 0001:0000eddc       ?SetRate@WaveStreamContext@@UAAKK@Z 1000fddc f   esai_common_topaz_v1:strmctxt.obj
 0001:0000eefc       ?Render@WaveStreamContext@@UAAPAEPAE00PAUTRANSFER_STATUS@@@Z 1000fefc f   esai_common_topaz_v1:strmctxt.obj
 0001:0000f090       ?ClearBuffer@StreamContext@@SAXPAE0@Z 10010090 f   esai_common_topaz_v1:strmctxt.obj
 0001:0000f0bc       ?GetProperty@StreamContext@@QAAKPAUtag_WAVEPROPINFO@@@Z 100100bc f   esai_common_topaz_v1:strmctxt.obj
 0001:0000f0fc       ?SetProperty@StreamContext@@QAAKPAUtag_WAVEPROPINFO@@@Z 100100fc f   esai_common_topaz_v1:strmctxt.obj
 0001:0000f13c       ??_EStreamContext@@UAAPAXI@Z 1001013c f i esai_common_topaz_v1:strmctxt.obj
 0001:0000f13c       ??_GStreamContext@@UAAPAXI@Z 1001013c f i esai_common_topaz_v1:strmctxt.obj
 0001:0000f180       ?COMPTYPE@@YAPAGK@Z        10010180 f   esai_common_topaz_v1:mixerdrv.obj
 0001:0000f220       ?LookupMxLine@@YAPBUtagMXLINEDESC@@G@Z 10010220 f   esai_common_topaz_v1:mixerdrv.obj
 0001:0000f2bc       ?PerformMixerCallbacks@@YAXKK@Z 100102bc f   esai_common_topaz_v1:mixerdrv.obj
 0001:0000f388       ?wdev_MXDM_GETDEVCAPS@@YAKPAUtagMIXERCAPS@@K@Z 10010388 f   esai_common_topaz_v1:mixerdrv.obj
 0001:0000f480       ?wdev_MXDM_OPEN@@YAKPAKPAUtMIXEROPENDESC@@K@Z 10010480 f   esai_common_topaz_v1:mixerdrv.obj
 0001:0000f5cc       ?wdev_MXDM_CLOSE@@YAKK@Z   100105cc f   esai_common_topaz_v1:mixerdrv.obj
 0001:0000f690       ?wdev_MXDM_GETLINEINFO@@YAKPAUtMIXERLINE@@K@Z 10010690 f   esai_common_topaz_v1:mixerdrv.obj
 0001:00010274       ?wdev_MXDM_GETLINECONTROLS@@YAKPAUtMIXERLINECONTROLS@@K@Z 10011274 f   esai_common_topaz_v1:mixerdrv.obj
 0001:00010970       ?wdev_MXDM_GETCONTROLDETAILS@@YAKPAUtMIXERCONTROLDETAILS@@K@Z 10011970 f   esai_common_topaz_v1:mixerdrv.obj
 0001:00010a8c       ?wdev_MXDM_SETCONTROLDETAILS@@YAKPAUtMIXERCONTROLDETAILS@@K@Z 10011a8c f   esai_common_topaz_v1:mixerdrv.obj
 0001:00010be0       ?InitMixerControls@@YAHXZ  10011be0 f   esai_common_topaz_v1:mixerdrv.obj
 0001:00010c58       ?HandleMixerMessage@@YAHPAUMMDRV_MESSAGE_PARAMS@@PAK@Z 10011c58 f   esai_common_topaz_v1:mixerdrv.obj
 0001:0001103c       ?SetMasterVolume@@YAIK@Z   1001203c f   esai_common_topaz_v1:mixerdrv.obj
 0001:000110bc       ?GetMasterVolume@@YAKXZ    100120bc f   esai_common_topaz_v1:mixerdrv.obj
 0001:00011110       ?LookupControlByIndex@MixerControlList@@QAAPAVMixerControl@@K@Z 10012110 f i esai_common_topaz_v1:mixerdrv.obj
 0001:00011168       ??0MixerControlList@@QAA@XZ 10012168 f i esai_common_topaz_v1:mixerdrv.obj
 0001:000112f0       ??0MixerControlVolumeMaster@@QAA@XZ 100122f0 f i esai_common_topaz_v1:mixerdrv.obj
 0001:00011334       ?SetControlID@MixerControl@@UAAXK@Z 10012334 f i esai_common_topaz_v1:mixerdrv.obj
 0001:00011358       ??0MixerControlVolume@@QAA@XZ 10012358 f i esai_common_topaz_v1:mixerdrv.obj
 0001:0001139c       ??0MixerControl@@QAA@XZ    1001239c f i esai_common_topaz_v1:mixerdrv.obj
 0001:000113e4       ?CopyMixerControl@MixerControl@@UAAXPAUtMIXERCONTROL@@@Z 100123e4 f i esai_common_topaz_v1:mixerdrv.obj
 0001:000114b8       ?GetControlID@MixerControl@@QAAKXZ 100124b8 f i esai_common_topaz_v1:mixerdrv.obj
 0001:000114e8       ?GetControlDetails@MixerControl@@UAAKPAUtMIXERCONTROLDETAILS@@K@Z 100124e8 f i esai_common_topaz_v1:mixerdrv.obj
 0001:00011510       ?SetControlDetails@MixerControl@@UAAKPAUtMIXERCONTROLDETAILS@@K@Z 10012510 f i esai_common_topaz_v1:mixerdrv.obj
 0001:00011538       ??_EMixerControl@@UAAPAXI@Z 10012538 f i esai_common_topaz_v1:mixerdrv.obj
 0001:00011538       ??_GMixerControl@@UAAPAXI@Z 10012538 f i esai_common_topaz_v1:mixerdrv.obj
 0001:0001157c       ??1MixerControl@@UAA@XZ    1001257c f i esai_common_topaz_v1:mixerdrv.obj
 0001:000115a0       ?CopyMixerControl@MixerControlVolume@@UAAXPAUtMIXERCONTROL@@@Z 100125a0 f i esai_common_topaz_v1:mixerdrv.obj
 0001:000116b4       ?GetControlType@MixerControlVolume@@UAAKXZ 100126b4 f i esai_common_topaz_v1:mixerdrv.obj
 0001:000116e0       ?GetControlDetails@MixerControlVolume@@UAAKPAUtMIXERCONTROLDETAILS@@K@Z 100126e0 f i esai_common_topaz_v1:mixerdrv.obj
 0001:000118b8       ?SetControlDetails@MixerControlVolume@@UAAKPAUtMIXERCONTROLDETAILS@@K@Z 100128b8 f i esai_common_topaz_v1:mixerdrv.obj
 0001:00011ac4       ??_EMixerControlVolume@@UAAPAXI@Z 10012ac4 f i esai_common_topaz_v1:mixerdrv.obj
 0001:00011ac4       ??_GMixerControlVolume@@UAAPAXI@Z 10012ac4 f i esai_common_topaz_v1:mixerdrv.obj
 0001:00011b08       ??1MixerControlVolume@@UAA@XZ 10012b08 f i esai_common_topaz_v1:mixerdrv.obj
 0001:00011b24       ?CopyMixerControl@MixerControlVolumeMaster@@UAAXPAUtMIXERCONTROL@@@Z 10012b24 f i esai_common_topaz_v1:mixerdrv.obj
 0001:00011b68       ?GetLineID@MixerControlVolumeMaster@@UAAGXZ 10012b68 f i esai_common_topaz_v1:mixerdrv.obj
 0001:00011b94       ?SetGain@MixerControlVolumeMaster@@UAAXK@Z 10012b94 f i esai_common_topaz_v1:mixerdrv.obj
 0001:00011bbc       ?GetGain@MixerControlVolumeMaster@@UAAKXZ 10012bbc f i esai_common_topaz_v1:mixerdrv.obj
 0001:00011bf8       ??_GMixerControlVolumeMaster@@UAAPAXI@Z 10012bf8 f i esai_common_topaz_v1:mixerdrv.obj
 0001:00011bf8       ??_EMixerControlVolumeMaster@@UAAPAXI@Z 10012bf8 f i esai_common_topaz_v1:mixerdrv.obj
 0001:00011c3c       ??1MixerControlVolumeMaster@@UAA@XZ 10012c3c f i esai_common_topaz_v1:mixerdrv.obj
 0001:00011c58       ??0MixerControlVolumeMic@@QAA@XZ 10012c58 f i esai_common_topaz_v1:mixerdrv.obj
 0001:00011c9c       ?CopyMixerControl@MixerControlVolumeMic@@UAAXPAUtMIXERCONTROL@@@Z 10012c9c f i esai_common_topaz_v1:mixerdrv.obj
 0001:00011ce0       ?GetLineID@MixerControlVolumeMic@@UAAGXZ 10012ce0 f i esai_common_topaz_v1:mixerdrv.obj
 0001:00011d0c       ?SetGain@MixerControlVolumeMic@@UAAXK@Z 10012d0c f i esai_common_topaz_v1:mixerdrv.obj
 0001:00011d34       ?GetGain@MixerControlVolumeMic@@UAAKXZ 10012d34 f i esai_common_topaz_v1:mixerdrv.obj
 0001:00011d70       ??_EMixerControlVolumeMic@@UAAPAXI@Z 10012d70 f i esai_common_topaz_v1:mixerdrv.obj
 0001:00011d70       ??_GMixerControlVolumeMic@@UAAPAXI@Z 10012d70 f i esai_common_topaz_v1:mixerdrv.obj
 0001:00011db4       ??1MixerControlVolumeMic@@UAA@XZ 10012db4 f i esai_common_topaz_v1:mixerdrv.obj
 0001:00011dd0       ??0MixerControlMuteMaster@@QAA@XZ 10012dd0 f i esai_common_topaz_v1:mixerdrv.obj
 0001:00011e14       ??0MixerControlBoolean@@QAA@XZ 10012e14 f i esai_common_topaz_v1:mixerdrv.obj
 0001:00011e58       ?CopyMixerControl@MixerControlBoolean@@UAAXPAUtMIXERCONTROL@@@Z 10012e58 f i esai_common_topaz_v1:mixerdrv.obj
 0001:00011f68       ?GetControlType@MixerControlBoolean@@UAAKXZ 10012f68 f i esai_common_topaz_v1:mixerdrv.obj
 0001:00011f94       ?GetControlDetails@MixerControlBoolean@@UAAKPAUtMIXERCONTROLDETAILS@@K@Z 10012f94 f i esai_common_topaz_v1:mixerdrv.obj
 0001:00012044       ?SetControlDetails@MixerControlBoolean@@UAAKPAUtMIXERCONTROLDETAILS@@K@Z 10013044 f i esai_common_topaz_v1:mixerdrv.obj
 0001:000120e8       ??_GMixerControlBoolean@@UAAPAXI@Z 100130e8 f i esai_common_topaz_v1:mixerdrv.obj
 0001:000120e8       ??_EMixerControlBoolean@@UAAPAXI@Z 100130e8 f i esai_common_topaz_v1:mixerdrv.obj
 0001:0001212c       ??1MixerControlBoolean@@UAA@XZ 1001312c f i esai_common_topaz_v1:mixerdrv.obj
 0001:00012148       ?CopyMixerControl@MixerControlMuteMaster@@UAAXPAUtMIXERCONTROL@@@Z 10013148 f i esai_common_topaz_v1:mixerdrv.obj
 0001:0001218c       ?GetControlType@MixerControlMuteMaster@@UAAKXZ 1001318c f i esai_common_topaz_v1:mixerdrv.obj
 0001:000121b8       ?GetLineID@MixerControlMuteMaster@@UAAGXZ 100131b8 f i esai_common_topaz_v1:mixerdrv.obj
 0001:000121e4       ?GetValue@MixerControlMuteMaster@@UAAHXZ 100131e4 f i esai_common_topaz_v1:mixerdrv.obj
 0001:00012220       ?SetValue@MixerControlMuteMaster@@UAAXH@Z 10013220 f i esai_common_topaz_v1:mixerdrv.obj
 0001:00012248       ??_GMixerControlMuteMaster@@UAAPAXI@Z 10013248 f i esai_common_topaz_v1:mixerdrv.obj
 0001:00012248       ??_EMixerControlMuteMaster@@UAAPAXI@Z 10013248 f i esai_common_topaz_v1:mixerdrv.obj
 0001:0001228c       ??1MixerControlMuteMaster@@UAA@XZ 1001328c f i esai_common_topaz_v1:mixerdrv.obj
 0001:000122a8       ??0MixerControlMuteMic@@QAA@XZ 100132a8 f i esai_common_topaz_v1:mixerdrv.obj
 0001:000122ec       ?CopyMixerControl@MixerControlMuteMic@@UAAXPAUtMIXERCONTROL@@@Z 100132ec f i esai_common_topaz_v1:mixerdrv.obj
 0001:00012330       ?GetLineID@MixerControlMuteMic@@UAAGXZ 10013330 f i esai_common_topaz_v1:mixerdrv.obj
 0001:0001235c       ?GetValue@MixerControlMuteMic@@UAAHXZ 1001335c f i esai_common_topaz_v1:mixerdrv.obj
 0001:00012398       ?SetValue@MixerControlMuteMic@@UAAXH@Z 10013398 f i esai_common_topaz_v1:mixerdrv.obj
 0001:000123c0       ??_GMixerControlMuteMic@@UAAPAXI@Z 100133c0 f i esai_common_topaz_v1:mixerdrv.obj
 0001:000123c0       ??_EMixerControlMuteMic@@UAAPAXI@Z 100133c0 f i esai_common_topaz_v1:mixerdrv.obj
 0001:00012404       ??1MixerControlMuteMic@@UAA@XZ 10013404 f i esai_common_topaz_v1:mixerdrv.obj
 0001:00012420       ??0MixerControlLoopback@@QAA@XZ 10013420 f i esai_common_topaz_v1:mixerdrv.obj
 0001:00012474       ?CopyMixerControl@MixerControlLoopback@@UAAXPAUtMIXERCONTROL@@@Z 10013474 f i esai_common_topaz_v1:mixerdrv.obj
 0001:000124bc       ?GetControlType@MixerControlLoopback@@UAAKXZ 100134bc f i esai_common_topaz_v1:mixerdrv.obj
 0001:000124e8       ?GetLineID@MixerControlLoopback@@UAAGXZ 100134e8 f i esai_common_topaz_v1:mixerdrv.obj
 0001:00012514       ?GetValue@MixerControlLoopback@@UAAHXZ 10013514 f i esai_common_topaz_v1:mixerdrv.obj
 0001:00012544       ?SetValue@MixerControlLoopback@@UAAXH@Z 10013544 f i esai_common_topaz_v1:mixerdrv.obj
 0001:00012558       ??_GMixerControlLoopback@@UAAPAXI@Z 10013558 f i esai_common_topaz_v1:mixerdrv.obj
 0001:00012558       ??_EMixerControlLoopback@@UAAPAXI@Z 10013558 f i esai_common_topaz_v1:mixerdrv.obj
 0001:0001259c       ??1MixerControlLoopback@@UAA@XZ 1001359c f i esai_common_topaz_v1:mixerdrv.obj
 0001:000125b8       ??0MixerControlInputMux@@QAA@XZ 100135b8 f i esai_common_topaz_v1:mixerdrv.obj
 0001:0001260c       ?CopyMixerControl@MixerControlInputMux@@UAAXPAUtMIXERCONTROL@@@Z 1001360c f i esai_common_topaz_v1:mixerdrv.obj
 0001:00012754       ?GetLineID@MixerControlInputMux@@UAAGXZ 10013754 f i esai_common_topaz_v1:mixerdrv.obj
 0001:00012780       ?GetControlType@MixerControlInputMux@@UAAKXZ 10013780 f i esai_common_topaz_v1:mixerdrv.obj
 0001:000127ac       ?GetNumSelections@MixerControlInputMux@@QAAKXZ 100137ac f i esai_common_topaz_v1:mixerdrv.obj
 0001:000127d4       ?GetControlDetails@MixerControlInputMux@@UAAKPAUtMIXERCONTROLDETAILS@@K@Z 100137d4 f i esai_common_topaz_v1:mixerdrv.obj
 0001:00012a24       ?GetListText@MixerControlInputMux@@QAAXPAUtMIXERCONTROLDETAILS_LISTTEXT@@K@Z 10013a24 f i esai_common_topaz_v1:mixerdrv.obj
 0001:00012b2c       ?GetComponentType@MixerControl@@QAAKXZ 10013b2c f i esai_common_topaz_v1:mixerdrv.obj
 0001:00012b94       ?GetCurrSelection@MixerControlInputMux@@QAAKK@Z 10013b94 f i esai_common_topaz_v1:mixerdrv.obj
 0001:00012be8       ?SetControlDetails@MixerControlInputMux@@UAAKPAUtMIXERCONTROLDETAILS@@K@Z 10013be8 f i esai_common_topaz_v1:mixerdrv.obj
 0001:00012d68       ?SetCurrSelection@MixerControlInputMux@@QAAXKH@Z 10013d68 f i esai_common_topaz_v1:mixerdrv.obj
 0001:00012de0       ??_EMixerControlInputMux@@UAAPAXI@Z 10013de0 f i esai_common_topaz_v1:mixerdrv.obj
 0001:00012de0       ??_GMixerControlInputMux@@UAAPAXI@Z 10013de0 f i esai_common_topaz_v1:mixerdrv.obj
 0001:00012e24       ??1MixerControlInputMux@@UAA@XZ 10013e24 f i esai_common_topaz_v1:mixerdrv.obj
 0001:00012e40       ??_GMixerControlList@@UAAPAXI@Z 10013e40 f i esai_common_topaz_v1:mixerdrv.obj
 0001:00012e40       ??_EMixerControlList@@UAAPAXI@Z 10013e40 f i esai_common_topaz_v1:mixerdrv.obj
 0001:00012e84       ??1MixerControlList@@UAA@XZ 10013e84 f i esai_common_topaz_v1:mixerdrv.obj
 0001:00012ef0       ?Open@InputStreamContext@@UAAKPAVDeviceContext@@PAUwaveopendesc_tag@@K@Z 10013ef0 f   esai_common_topaz_v1:input.obj
 0001:00012f54       ?DoCallbackReturnBuffer@InputStreamContext@@UAAXPAUwavehdr_tag@@@Z 10013f54 f   esai_common_topaz_v1:input.obj
 0001:00012f7c       ?DoCallbackStreamOpened@InputStreamContext@@UAAXXZ 10013f7c f   esai_common_topaz_v1:input.obj
 0001:00012fa8       ?DoCallbackStreamClosed@InputStreamContext@@UAAXXZ 10013fa8 f   esai_common_topaz_v1:input.obj
 0001:00012fd4       ?Stop@InputStreamContext@@UAAKXZ 10013fd4 f   esai_common_topaz_v1:input.obj
 0001:0001303c       ?Render2@InputStreamContext@@UAAPAEPAE00PAUTRANSFER_STATUS@@@Z 1001403c f   esai_common_topaz_v1:input.obj
 0001:00013458       ?ResetBaseInfo@InputStreamContext@@UAAXXZ 10014458 f   esai_common_topaz_v1:input.obj
 0001:0001346c       ?Render2@InputStreamContextEx@@UAAPAEPAE00PAUTRANSFER_STATUS@@@Z 1001446c f   esai_common_topaz_v1:input.obj
 0001:00013558       ?Open@OutputStreamContext@@UAAKPAVDeviceContext@@PAUwaveopendesc_tag@@K@Z 10014558 f   esai_common_topaz_v1:output.obj
 0001:000135f0       ?Reset@OutputStreamContext@@UAAKXZ 100145f0 f   esai_common_topaz_v1:output.obj
 0001:00013654       ?ResetBaseInfo@OutputStreamContext@@UAAXXZ 10014654 f   esai_common_topaz_v1:output.obj
 0001:00013668       ?Render2@OutputStreamContextM8@@UAAPAEPAE00PAUTRANSFER_STATUS@@@Z 10014668 f   esai_common_topaz_v1:output.obj
 0001:000139d8       ?Render2@OutputStreamContextM16@@UAAPAEPAE00PAUTRANSFER_STATUS@@@Z 100149d8 f   esai_common_topaz_v1:output.obj
 0001:00013d38       ?Render2@OutputStreamContextS8@@UAAPAEPAE00PAUTRANSFER_STATUS@@@Z 10014d38 f   esai_common_topaz_v1:output.obj
 0001:0001413c       ?Render2@OutputStreamContextS16@@UAAPAEPAE00PAUTRANSFER_STATUS@@@Z 1001513c f   esai_common_topaz_v1:output.obj
 0001:00014520       ?Render2@OutputStreamContextMC@@UAAPAEPAE00PAUTRANSFER_STATUS@@@Z 10015520 f   esai_common_topaz_v1:output.obj
 0001:00014b9c       ?Render2@OutputStreamContextEx@@UAAPAEPAE00PAUTRANSFER_STATUS@@@Z 10015b9c f   esai_common_topaz_v1:output.obj
 0001:00014c88       ?GetESAIBaseRegAddr@@YAII@Z 10015c88 f   esai_mx25_topaz_v1:mx25esai.obj
 0001:00014cb4       ?GetSdmaChannelIRQ@@YAKI@Z 10015cb4 f   esai_mx25_topaz_v1:mx25esai.obj
 0001:00014ce0       AsrcInit                   10015ce0 f   asrcbase_mx25_topaz_v1_stub:mx25asrc_stub.obj
 0001:00014d08       AsrcDeinit                 10015d08 f   asrcbase_mx25_topaz_v1_stub:mx25asrc_stub.obj
 0001:00014d20       AsrcOpenPair               10015d20 f   asrcbase_mx25_topaz_v1_stub:mx25asrc_stub.obj
 0001:00014d48       AsrcStartConv              10015d48 f   asrcbase_mx25_topaz_v1_stub:mx25asrc_stub.obj
 0001:00014d70       AsrcStopConv               10015d70 f   asrcbase_mx25_topaz_v1_stub:mx25asrc_stub.obj
 0001:00014d98       AsrcGetInputBufStatus      10015d98 f   asrcbase_mx25_topaz_v1_stub:mx25asrc_stub.obj
 0001:00014dc0       AsrcClosePair              10015dc0 f   asrcbase_mx25_topaz_v1_stub:mx25asrc_stub.obj
 0001:00014dd4       AsrcSetP2PDeviceWML        10015dd4 f   asrcbase_mx25_topaz_v1_stub:mx25asrc_stub.obj
 0001:00014dfc       AsrcConfigPair             10015dfc f   asrcbase_mx25_topaz_v1_stub:mx25asrc_stub.obj
 0001:00014e24       AsrcSetOutputBuf           10015e24 f   asrcbase_mx25_topaz_v1_stub:mx25asrc_stub.obj
 0001:00014e4c       AsrcSetInputBuf            10015e4c f   asrcbase_mx25_topaz_v1_stub:mx25asrc_stub.obj
 0001:00014e74       NKDbgPrintfW               10015e74 f   coredll:COREDLL.dll
 0001:00014e84       GetLastError               10015e84 f   coredll:COREDLL.dll
 0001:00014e94       CloseHandle                10015e94 f   coredll:COREDLL.dll
 0001:00014ea4       Sleep                      10015ea4 f   coredll:COREDLL.dll
 0001:00014eb4       RegCloseKey                10015eb4 f   coredll:COREDLL.dll
 0001:00014ec4       RegQueryValueExW           10015ec4 f   coredll:COREDLL.dll
 0001:00014ed4       RegOpenKeyExW              10015ed4 f   coredll:COREDLL.dll
 0001:00014ee4       DisableThreadLibraryCalls  10015ee4 f   coredll:COREDLL.dll
 0001:00014ef4       RegisterDbgZones           10015ef4 f   coredll:COREDLL.dll
 0001:00014f04       SetLastError               10015f04 f   coredll:COREDLL.dll
 0001:00014f14       EnterCriticalSection       10015f14 f   coredll:COREDLL.dll
 0001:00014f24       LeaveCriticalSection       10015f24 f   coredll:COREDLL.dll
 0001:00014f34       CeGetCallerTrust           10015f34 f   coredll:COREDLL.dll
 0001:00014f44       InitializeCriticalSection  10015f44 f   coredll:COREDLL.dll
 0001:00014f54       DeleteCriticalSection      10015f54 f   coredll:COREDLL.dll
 0001:00014f64       EventModify                10015f64 f   coredll:COREDLL.dll
 0001:00014f74       KernelIoControl            10015f74 f   coredll:COREDLL.dll
 0001:00014f84       CeSetThreadPriority        10015f84 f   coredll:COREDLL.dll
 0001:00014f94       CreateThread               10015f94 f   coredll:COREDLL.dll
 0001:00014fa4       InterruptInitialize        10015fa4 f   coredll:COREDLL.dll
 0001:00014fb4       CreateEventW               10015fb4 f   coredll:COREDLL.dll
 0001:00014fc4       WaitForSingleObject        10015fc4 f   coredll:COREDLL.dll
 0001:00014fd4       WaitForMultipleObjects     10015fd4 f   coredll:COREDLL.dll
 0001:00014fe4       OpenDeviceKey              10015fe4 f   coredll:COREDLL.dll
 0001:00014ff4       RegSetValueExW             10015ff4 f   coredll:COREDLL.dll
 0001:00015004       CeSafeCopyMemory           10016004 f   coredll:COREDLL.dll
 0001:00015014       LocalAlloc                 10016014 f   coredll:COREDLL.dll
 0001:00015024       LocalFree                  10016024 f   coredll:COREDLL.dll
 0001:00015034       HalAllocateCommonBuffer    10016034 f   ceddk:CEDDK.dll
 0001:00015044       HalFreeCommonBuffer        10016044 f   ceddk:CEDDK.dll
 0001:00015054       MmMapIoSpace               10016054 f   ceddk:CEDDK.dll
 0001:00015064       MmUnmapIoSpace             10016064 f   ceddk:CEDDK.dll
 0001:00015074       DDKGpioWriteDataPin        10016074 f   cspddk:CSPDDK.dll
 0001:00015084       DDKIomuxSetPinMux          10016084 f   cspddk:CSPDDK.dll
 0001:00015094       DDKClockSetGatingMode      10016094 f   cspddk:CSPDDK.dll
 0001:000150a4       DDKSdmaAllocChain          100160a4 f   cspddk:CSPDDK.dll
 0001:000150b4       DDKSdmaOpenChan            100160b4 f   cspddk:CSPDDK.dll
 0001:000150c4       DDKSdmaSetBufDesc          100160c4 f   cspddk:CSPDDK.dll
 0001:000150d4       DDKSdmaStartChan           100160d4 f   cspddk:CSPDDK.dll
 0001:000150e4       DDKSdmaInitChain           100160e4 f   cspddk:CSPDDK.dll
 0001:000150f4       DDKSdmaStopChan            100160f4 f   cspddk:CSPDDK.dll
 0001:00015104       DDKSdmaClearBufDescStatus  10016104 f   cspddk:CSPDDK.dll
 0001:00015114       DDKSdmaGetChainStatus      10016114 f   cspddk:CSPDDK.dll
 0001:00015124       timeSetEvent               10016124 f   mmtimer:MMTimer.dll
 0001:00015134       timeKillEvent              10016134 f   mmtimer:MMTimer.dll
 0001:00015144       CSPIOpenHandle             10016144 f   spisdk_common_topaz_v1:spisdk.obj
 0001:00015260       CSPICloseHandle            10016260 f   spisdk_common_topaz_v1:spisdk.obj
 0001:0001535c       CSPIExchange               1001635c f   spisdk_common_topaz_v1:spisdk.obj
 0001:0001547c       CSPIEnableLoopback         1001647c f   spisdk_common_topaz_v1:spisdk.obj
 0001:0001559c       CSPIDisableLoopback        1001659c f   spisdk_common_topaz_v1:spisdk.obj
 0001:000156bc       DllEntry                   100166bc f   spisdk_common_topaz_v1:spisdk.obj
 0001:00015784       I2CCloseHandle             10016784 f   i2csdk:I2CSDK.dll
 0001:00015794       I2CSetMasterMode           10016794 f   i2csdk:I2CSDK.dll
 0001:000157a4       I2COpenHandle              100167a4 f   i2csdk:I2CSDK.dll
 0001:000157b4       I2CTransfer                100167b4 f   i2csdk:I2CSDK.dll
 0001:000157c4       ??2@YAPAXI@Z               100167c4 f   corelib1:COREDLL.dll
 0001:000157d4       ??3@YAXPAX@Z               100167d4 f   corelib1:COREDLL.dll
 0001:000157e4       memset                     100167e4 f   corelib1:COREDLL.dll
 0001:000157f4       __C_specific_handler       100167f4 f   corelib1:COREDLL.dll
 0001:00015804       __rt_sdiv                  10016804 f   corelib1:COREDLL.dll
 0001:00015814       memcpy                     10016814 f   corelib1:COREDLL.dll
 0001:00015824       __rt_udiv                  10016824 f   corelib1:COREDLL.dll
 0001:00015834       _purecall                  10016834 f   corelib1:COREDLL.dll
 0001:00015844       __rt_sdiv64by64            10016844 f   corelib1:COREDLL.dll
 0001:00015854       memcmp                     10016854 f   corelib1:COREDLL.dll
 0001:00015864       wcscpy                     10016864 f   corelib1:COREDLL.dll
 0001:00015874       CreateFileW                10016874 f   coredll:COREDLL.dll
 0001:00015884       DeviceIoControl            10016884 f   coredll:COREDLL.dll
 0001:000158d0       __IMPORT_DESCRIPTOR_COREDLL 100168d0     coredll:COREDLL.dll
 0001:000158e4       __IMPORT_DESCRIPTOR_CEDDK  100168e4     ceddk:CEDDK.dll
 0001:000158f8       __IMPORT_DESCRIPTOR_CSPDDK 100168f8     cspddk:CSPDDK.dll
 0001:0001590c       __IMPORT_DESCRIPTOR_MMTimer 1001690c     mmtimer:MMTimer.dll
 0001:00015920       __IMPORT_DESCRIPTOR_I2CSDK 10016920     i2csdk:I2CSDK.dll
 0001:00015934       __NULL_IMPORT_DESCRIPTOR   10016934     coredll:COREDLL.dll
 0002:00000000       __imp_MmMapIoSpace         10017000     ceddk:CEDDK.dll
 0002:00000004       __imp_HalFreeCommonBuffer  10017004     ceddk:CEDDK.dll
 0002:00000008       __imp_HalAllocateCommonBuffer 10017008     ceddk:CEDDK.dll
 0002:0000000c       __imp_MmUnmapIoSpace       1001700c     ceddk:CEDDK.dll
 0002:00000010       \177CEDDK_NULL_THUNK_DATA  10017010     ceddk:CEDDK.dll
 0002:00000014       __imp_RegQueryValueExW     10017014     coredll:COREDLL.dll
 0002:00000018       __imp_RegOpenKeyExW        10017018     coredll:COREDLL.dll
 0002:0000001c       __imp_DisableThreadLibraryCalls 1001701c     coredll:COREDLL.dll
 0002:00000020       __imp_RegisterDbgZones     10017020     coredll:COREDLL.dll
 0002:00000024       __imp_SetLastError         10017024     coredll:COREDLL.dll
 0002:00000028       __imp_EnterCriticalSection 10017028     coredll:COREDLL.dll
 0002:0000002c       __imp_LeaveCriticalSection 1001702c     coredll:COREDLL.dll
 0002:00000030       __imp_CeGetCallerTrust     10017030     coredll:COREDLL.dll
 0002:00000034       __imp_InitializeCriticalSection 10017034     coredll:COREDLL.dll
 0002:00000038       __imp_DeleteCriticalSection 10017038     coredll:COREDLL.dll
 0002:0000003c       __imp_EventModify          1001703c     coredll:COREDLL.dll
 0002:00000040       __imp_RegCloseKey          10017040     coredll:COREDLL.dll
 0002:00000044       __imp_CeSetThreadPriority  10017044     coredll:COREDLL.dll
 0002:00000048       __imp_CreateThread         10017048     coredll:COREDLL.dll
 0002:0000004c       __imp_InterruptInitialize  1001704c     coredll:COREDLL.dll
 0002:00000050       __imp_CreateEventW         10017050     coredll:COREDLL.dll
 0002:00000054       __imp_WaitForSingleObject  10017054     coredll:COREDLL.dll
 0002:00000058       __imp_WaitForMultipleObjects 10017058     coredll:COREDLL.dll
 0002:0000005c       __imp_OpenDeviceKey        1001705c     coredll:COREDLL.dll
 0002:00000060       __imp_RegSetValueExW       10017060     coredll:COREDLL.dll
 0002:00000064       __imp_CeSafeCopyMemory     10017064     coredll:COREDLL.dll
 0002:00000068       __imp_LocalAlloc           10017068     coredll:COREDLL.dll
 0002:0000006c       __imp_LocalFree            1001706c     coredll:COREDLL.dll
 0002:00000070       __imp_Sleep                10017070     coredll:COREDLL.dll
 0002:00000074       __imp_CloseHandle          10017074     coredll:COREDLL.dll
 0002:00000078       __imp_GetLastError         10017078     coredll:COREDLL.dll
 0002:0000007c       __imp_KernelIoControl      1001707c     coredll:COREDLL.dll
 0002:00000080       __imp_NKDbgPrintfW         10017080     coredll:COREDLL.dll
 0002:00000084       __imp_CreateFileW          10017084     coredll:COREDLL.dll
 0002:00000088       __imp_wcscpy               10017088     corelib1:COREDLL.dll
 0002:0000008c       __imp_memcmp               1001708c     corelib1:COREDLL.dll
 0002:00000090       __imp___rt_sdiv64by64      10017090     corelib1:COREDLL.dll
 0002:00000094       __imp__purecall            10017094     corelib1:COREDLL.dll
 0002:00000098       __imp___rt_udiv            10017098     corelib1:COREDLL.dll
 0002:0000009c       __imp_memcpy               1001709c     corelib1:COREDLL.dll
 0002:000000a0       __imp___rt_sdiv            100170a0     corelib1:COREDLL.dll
 0002:000000a4       __imp___C_specific_handler 100170a4     corelib1:COREDLL.dll
 0002:000000a8       __imp_memset               100170a8     corelib1:COREDLL.dll
 0002:000000ac       __imp_??3@YAXPAX@Z         100170ac     corelib1:COREDLL.dll
 0002:000000b0       __imp_??2@YAPAXI@Z         100170b0     corelib1:COREDLL.dll
 0002:000000b4       __imp_DeviceIoControl      100170b4     coredll:COREDLL.dll
 0002:000000b8       \177COREDLL_NULL_THUNK_DATA 100170b8     coredll:COREDLL.dll
 0002:000000bc       __imp_DDKGpioWriteDataPin  100170bc     cspddk:CSPDDK.dll
 0002:000000c0       __imp_DDKIomuxSetPinMux    100170c0     cspddk:CSPDDK.dll
 0002:000000c4       __imp_DDKClockSetGatingMode 100170c4     cspddk:CSPDDK.dll
 0002:000000c8       __imp_DDKSdmaAllocChain    100170c8     cspddk:CSPDDK.dll
 0002:000000cc       __imp_DDKSdmaOpenChan      100170cc     cspddk:CSPDDK.dll
 0002:000000d0       __imp_DDKSdmaSetBufDesc    100170d0     cspddk:CSPDDK.dll
 0002:000000d4       __imp_DDKSdmaStartChan     100170d4     cspddk:CSPDDK.dll
 0002:000000d8       __imp_DDKSdmaGetChainStatus 100170d8     cspddk:CSPDDK.dll
 0002:000000dc       __imp_DDKSdmaClearBufDescStatus 100170dc     cspddk:CSPDDK.dll
 0002:000000e0       __imp_DDKSdmaStopChan      100170e0     cspddk:CSPDDK.dll
 0002:000000e4       __imp_DDKSdmaInitChain     100170e4     cspddk:CSPDDK.dll
 0002:000000e8       \177CSPDDK_NULL_THUNK_DATA 100170e8     cspddk:CSPDDK.dll
 0002:000000ec       __imp_I2CTransfer          100170ec     i2csdk:I2CSDK.dll
 0002:000000f0       __imp_I2COpenHandle        100170f0     i2csdk:I2CSDK.dll
 0002:000000f4       __imp_I2CSetMasterMode     100170f4     i2csdk:I2CSDK.dll
 0002:000000f8       __imp_I2CCloseHandle       100170f8     i2csdk:I2CSDK.dll
 0002:000000fc       \177I2CSDK_NULL_THUNK_DATA 100170fc     i2csdk:I2CSDK.dll
 0002:00000100       __imp_timeKillEvent        10017100     mmtimer:MMTimer.dll
 0002:00000104       __imp_timeSetEvent         10017104     mmtimer:MMTimer.dll
 0002:00000108       \177MMTimer_NULL_THUNK_DATA 10017108     mmtimer:MMTimer.dll
 0002:00000120       ?ctype_table@@3PAUMMSYSCODE@@A 10017120     esai_common_topaz_v1:mixerdrv.obj
 0002:00000210       ?szNames@?1??GetListText@MixerControlInputMux@@QAAXPAUtMIXERCONTROLDETAILS_LISTTEXT@@K@Z@4PAPBGA 10017210     esai_common_topaz_v1:mixerdrv.obj
 0002:00000218       dpCurSettings              10017218     spisdk_common_topaz_v1:spisdk.obj
 0002:00000664       ?g_pHWContext@@3PAVHardwareContext@@A 10017664     esai_common_topaz_v1:hwctxt.obj

 entry point at        0001:000156bc

 Static symbols

